:0200000480007A
:10000000B72F0000938F0F8073900F306F00400365
:100010001300000013000000130000001300000094
:100020001300000013000000130000001300000084
:100030001300000013000000130000001300000074
:100040009702000093824211739052309300000097
:10005000130100009301000013020000930200004E
:100060001303000093030000130400009304000036
:10007000130500009305000013060000930600001E
:100080001307000093070000130800009308000006
:100090001309000093090000130A0000930A0000EE
:1000A000130B0000930B0000130C0000930C0000D6
:1000B000130D0000930D0000130E0000930E0000BE
:1000C000130F0000930F000097110200938141B2BB
:1000D00017050200130505339795030093854564C2
:1000E00013060000EF00001A170502001305852F04
:1000F000970502009385852F13060000EF008018F6
:1001000017A503001305056297B5030093854561A4
:1001100037B6ABAB1306B6BAEF00C01617B1030083
:1001200013014160EF70006F9392120093D212009E
:100130009382D2FF638A02008322010013014100EF
:100140006F0000177300203083220100130141006B
:10015000730020301301C1FF23205100F32220340B
:10016000E3C402FC8322010013014100130141F8A2
:1001700023221100232421002326310023284100BB
:10018000232A5100232C6100232E71002320810299
:10019000232291022324A1022326B1022328C10293
:1001A000232AD102232CE102232EF1022320010570
:1001B0002322110523242105232631052328410567
:1001C000232A5105232C6105232E71052320810745
:1001D000232291072324A1072326B1072328C1073F
:1001E000232AD107232CE107232EF107732520347E
:1001F000F3251034130601006F000000731015344E
:1002000083204100032181008321C10003220101D9
:1002100083224101032381018323C10103240102BD
:1002200083244102032581028325C10203260103A1
:1002300083264103032781038327C1030328010485
:1002400083284104032981048329C104032A010569
:10025000832A4105032B8105832BC105032C01064D
:10026000832C4106032D8106832DC106032E010731
:10027000832E4107032F8107832FC1071301C10775
:10028000730020302320C5006376B50013054500B8
:100290006FF05FFF678000000000000000000000BA
:1002A000000000000000000000000000000000004E
:1002B000130101F8232011002322210023243100FF
:1002C0002326410023285100232A6100232C71009A
:1002D000232E8100232091022322A1022324B10294
:1002E0002326C1022328D102232AE102232CF10272
:1002F000232E010323201105232221052324310568
:100300002326410523285105232A6105232C710545
:10031000232E8105232091072322A1072324B1073F
:100320002326C1072328D107232AE107232CF1071D
:100330009702020083A2020B23A02200F3221034B2
:10034000232E5106EF008046170102000321810988
:10035000032101008322C10773901234B7220000E9
:100360009382028873A00230832001000322C1001F
:100370008322010103234101832381010324C1015D
:100380008324010203254102832581020326C10241
:100390008326010303274103832781030328C10325
:1003A000832801040329410483298104032AC10409
:1003B000832A0105032B4105832B8105032CC105ED
:1003C000832C0106032D4106832D8106032EC106D1
:1003D000832E0107032F4107832F81071301010893
:1003E00073002030970202009382C20123A0120002
:1003F00023A2220023A4320023A6420023A85200F5
:1004000023AA620023AC720023AE820023A09202D2
:1004100023A2A20223A4B20223A6C20223A8D202CC
:1004200023AAE20223ACF20223AE020323A01205A8
:1004300023A2220523A4320523A6420523A85205A0
:1004400023AA620523AC720523AE820523A092077E
:1004500023A2A20723A4B20723A6C20723A8D20778
:1004600023AAE20723ACF207EF700029170102006C
:10047000032141F7032101008322C1077390123445
:10048000B72200009382028873A00230832001000B
:100490000322C1008322010103234101832381013F
:1004A0000324C10183240102032541028325810223
:1004B0000326C10283260103032741038327810307
:1004C0000328C103832801040329410483298104EB
:1004D000032AC104832A0105032B4105832B8105CF
:1004E000032CC105832C0106032D4106832D8106B3
:1004F000032EC106832E0107032F4107832F810797
:10050000130101087300203097020200938282EFEA
:1005100083A0020003A1420083A1820003A2C200C3
:1005200083A2020103A3420183A3820103A4C201A7
:1005300083A4020203A5420283A5820203A6C2028B
:1005400083A6020303A7420383A7820303A8C2036F
:1005500083A8020403A9420483A9820403AAC20453
:1005600083AA020503AB420583AB820503ACC20537
:1005700083AC020603AD420683AD820603AEC2061B
:1005800083AE020703AFC20983AF82076780000012
:1005900073700430130101F823201100232221007D
:1005A000232431002326410023285100232A6100FF
:1005B000232C7100232E8100232091022322A102EB
:1005C0002324B1022326C1022328D102232AE102D7
:1005D000232CF102232E01032320110523222105C0
:1005E000232431052326410523285105232A6105AB
:1005F000232C7105232E8105232091072322A10797
:100600002324B1072326C1072328D107232AE10782
:10061000232CF1079702020083A2C2DC23A0220050
:10062000232E1106EF30000F17010200032181DB9A
:10063000032101008322C10773901234B722000006
:100640009382028873A00230832001000322C1003C
:100650008322010103234101832381010324C1017A
:100660008324010203254102832581020326C1025E
:100670008326010303274103832781030328C10342
:10068000832801040329410483298104032AC10426
:10069000832A0105032B4105832B8105032CC1050A
:1006A000832C0106032D4106832D8106032EC106EE
:1006B000832E0107032F4107832F810713010108B0
:1006C0007300203097070200938787D203A70700A3
:1006D0009307F0FF6306F700737004306F000000AB
:1006E000737004306F000000130101FF2326A10086
:1006F0008327C100739047301300000013010101EC
:1007000067800000130101FFF32740302326F1002A
:1007100073F043308327C1001385070013010101E3
:1007200067800000130101FF2326A1002324B100EC
:100730002322C1008327C1009387C7FF2326F1002E
:10074000032781008327C10023A0E7008327C1007E
:10075000938787FA2326F100032741008327C100EE
:1007600023A0E7008327C100938787FE2326F1009B
:1007700093870100138707008327C10023A0E700A8
:100780008327C100938747FF2326F1001707000046
:10079000130787F38327C10023A0E7008327C10045
:1007A000138507001301010167800000130101FF99
:1007B00023261100EF60106AEF20504C93070500CC
:1007C00063840700EF201075130000008320C10030
:1007D0001301010167800000130101FF2326A1001E
:1007E0008327C100138787008327C10023A2E70066
:1007F0008327C1001307F0FF23A4E7008327C1006C
:10080000138787008327C10023A6E7008327C10041
:10081000138787008327C10023A8E7008327C1002F
:1008200023A00700130000001301010167800000EE
:10083000130101FF2326A1008327C10023A807007D
:10084000130000001301010167800000130101FE85
:100850002326A1002324B1008327C10083A74700DA
:10086000232EF100832781000327C10123A2E70083
:100870008327C10103A787008327810023A4E70002
:100880008327C10183A787000327810023A2E700F4
:100890008327C1010327810023A4E7008327810068
:1008A0000327C10023A8E7008327C10083A707000F
:1008B000138717008327C10023A0E700130000005F
:1008C0001301010267800000130101FE2326A1002D
:1008D0002324B1008327810083A70700232CF10084
:1008E000032781019307F0FF631AF7008327C100F4
:1008F00083A70701232EF1006F0040038327C10067
:1009000093878700232EF1006F0000018327C10128
:1009100083A74700232EF1008327C10183A7470047
:1009200083A7070003278101E372F7FE8327C10134
:1009300003A747008327810023A2E70083278100C4
:1009400083A747000327810023A4E70083278100B2
:100950000327C10123A4E7008327C10103278100E6
:1009600023A2E700832781000327C10023A8E70013
:100970008327C10083A70700138717008327C100BF
:1009800023A0E700130000001301010267800000AC
:10099000130101FE2326A1008327C10083A70701BD
:1009A000232EF1008327C10083A747000327C1003E
:1009B0000327870023A4E7008327C10083A78700BC
:1009C0000327C1000327470023A2E7008327C101B3
:1009D00083A747000327C100631AF7008327C100DC
:1009E00003A787008327C10123A2E7008327C10053
:1009F00023A807008327C10183A707001387F7FFF8
:100A00008327C10123A0E7008327C10183A7070033
:100A1000138507001301010267800000130101FD27
:100A200023261102232481022326A1002324B100BE
:100A30008327C100232EF1008327C101639607009D
:100A4000737004306F000000EF3050778327C101CE
:100A500003A407008327C10103A7C7038327C1019C
:100A600083A707049385070013050700EF80802CF8
:100A7000930705003307F4008327C10123A2E70091
:100A80008327C10123AC07028327C10103A7070005
:100A90008327C10123A4E7008327C10103A4070022
:100AA0008327C10183A7C7031387F7FF8327C101EA
:100AB00083A707049385070013050700EF808027AD
:100AC000930705003307F4008327C10123A6E7003D
:100AD0008327C1011307F0FF23A2E7048327C10185
:100AE0001307F0FF23A4E70483278100639A07021A
:100AF0008327C10183A70701638407048327C101FA
:100B00009387070113850700EF3080021307050064
:100B1000930710006316F702EFF09FA76F004002E3
:100B20008327C1019387070113850700EFF0DFCA10
:100B30008327C1019387470213850700EFF0DFC9C0
:100B4000EF30D06B93071000138507008320C1029C
:100B5000032481021301010367800000130101FDDA
:100B6000232611022326A1002324B10093070600A7
:100B7000A303F100232C01008327C1006396070023
:100B8000737004306F0000008327810063960700B4
:100B9000232E01006F00C001832581000325C100C1
:100BA000EF8040199307050093871700232EF1006B
:100BB0008327C1019387470513850700EF50502411
:100BC000232AA1008327410163820706832781002E
:100BD000639A0700832741010327410123A0E7000F
:100BE0006F00400183274101138747058327410197
:100BF00023A0E700832741010327C10023AEE702BA
:100C0000832741010327810023A0E70493051000F7
:100C100003254101EFF09FE0832741010347710065
:100C20002388E70483274101232CF10083278101D6
:100C300063960700737004306F0000008327810102
:100C4000138507008320C1021301010367800000A0
:100C5000130101FD2326110293070500A307F100EC
:100C600013054005EF50D019232EA1008327C101A1
:100C7000638C07088327C10123A207008327C101D2
:100C800023A007008327C10123A407008327C101F4
:100C900023A607008327C10123AC07028327C101D4
:100CA0001307100023AEE7028327C10123A0070426
:100CB0008327C1011307F0FF23A2E7048327C101A3
:100CC0001307F0FF23A4E7048327C1010347F100C2
:100CD0002388E7048327C101938707011385070051
:100CE000EFF09FAF8327C101938747021385070069
:100CF000EFF09FAE9306000013060000930500007E
:100D00000325C101EF00001E8327C10113850700E1
:100D10008320C1021301010367800000130101FD5C
:100D200023261102232481022326A1008327C10048
:100D3000232CF10083278101639607007370043030
:100D40006F0000008327810103A44700EF30501695
:100D5000930705006312F4048327810183A7C7006A
:100D60001387F7FF8327810123A6E70083278101EB
:100D700083A7C700639C07009306000013060000CA
:100D80009305000003258101EF00C01593071000B3
:100D9000232EF1006F008000232E01008327C10164
:100DA000138507008320C10203248102130101037C
:100DB00067800000130101FD232611022324810214
:100DC0002326A1002324B1008327C100232CF10096
:100DD0008327810163960700737004306F00000061
:100DE0008327810103A44700EF30900C930705008F
:100DF0006312F4028327810183A7C70013871700BA
:100E00008327810123A6E70093071000232EF1001A
:100E10006F00C003930600000326810093050000C5
:100E200003258101EF00100F232EA1000327C1012C
:100E300093071000631CF7008327810183A7C70075
:100E4000138717008327810123A6E7008327C101A9
:100E5000138507008320C1020324810213010103CB
:100E600067800000130101FD232611022326A10043
:100E70002324B1008327C1006396070073700430F8
:100E80006F000000032781008327C10063F6E7009D
:100E9000737004306F0000001306200093050000FB
:100EA0000325C100EFF09FCB232EA1008327C101B2
:100EB000638807008327C1010327810023ACE70271
:100EC0008327C10163960700737004306F00000030
:100ED0008327C101138507008320C1021301010389
:100EE00067800000130101FC232E11022326A100BC
:100EF0002324B1002322C1002320D1002326010294
:100F00008327C1002324F10283278102639607000F
:100F1000737004306F00000083278100639807001E
:100F20008327810283A707046396070093071000B5
:100F30006F00800093070000639607007370043011
:100F40006F0000000327010093072000631AF700D9
:100F50008327810203A7C703930710006316F700D6
:100F6000930710006F00800093070000639607004E
:100F7000737004306F000000EF30C07593070500F8
:100F800063960700832741006396070093071000CC
:100F90006F008000930700006396070073700430B1
:100FA0006F000000EF3090218327810203A78703A1
:100FB0008327810283A7C7036368F7000327010023
:100FC000930720006310F7060326010083258100A4
:100FD00003258102EF0050522322A10283278102C0
:100FE00083A747026384070283278102938747020E
:100FF00013850700EF20D033130705009307100077
:10100000631CF700EFF0CFD86F0000018327410287
:1010100063840700EFF0CFD7EF30501E9307100026
:101020006F00400F8327410063980700EF30101DC9
:10103000930700006F00000E8327C102639C070026
:101040009307C10113850700EF2090539307100009
:101050002326F102EF30901AEF200000EF30101637
:101060008327810203A747049307F0FF6316F70065
:101070008327810223A207048327810203A7870411
:101080009307F0FF6316F7008327810223A4070468
:10109000EF30D016130741009307C10193050700F5
:1010A00013850700EF20905293070500639C070407
:1010B00003258102EF00907C93070500638C0702F3
:1010C00083278102938707010327410093050700C7
:1010D00013850700EF20500003258102EF00D06246
:1010E000EF10D07993070500E39E07EAEFF04FCAAF
:1010F0006FF05FEB03258102EF001061EF101078B5
:101100006FF05FEA03258102EF001060EF101077A7
:1011100093070000138507008320C1031301010416
:1011200067800000130101FD232611022326A10080
:101130002324B1002322C1002320D100232E01004B
:101140008327C100232CF1008327810163960700C8
:10115000737004306F0000008327810063980700DC
:101160008327810183A70704639607009307100074
:101170006F008000930700006396070073700430CF
:101180006F000000EF3090038327810103A78703DE
:101190008327810183A7C7036376F7040326010031
:1011A0008325810003258101EF001035832781010C
:1011B00083A747026382070283278101938747023F
:1011C00013850700EF20D0161307050093071000C2
:1011D0006314F700EFF0CFBBEF305002930710001D
:1011E0006F00C0098327410063980700EF301001AA
:1011F000930700006F0080088327C101639C0700EC
:101200009307010113850700EF2090379307100023
:10121000232EF100EF30807EEF30407A130741003B
:10122000930701019305070013850700EF20103A8B
:1012300093070500639A070203258101EF001064FC
:1012400093070500638807028327810193870701BD
:10125000032741009305070013850700EF20C067AF
:10126000EFF00FB36F000001EF30407993070000FB
:101270006F00C000EF3080786FF0DFF0138507005B
:101280008320C1021301010367800000130101FCE8
:10129000232E11022326A1002324B1002322C10002
:1012A0002320D100232601028327C1002324F10239
:1012B0008327810263960700737004306F0000007B
:1012C00083278100639807008327810283A707048F
:1012D00063960700930710006F00800093070000DB
:1012E00063960700737004306F000000EF30006DEC
:1012F0008327810283A787036382070C83278102E8
:1013000083A7C7002322F1028325810003258102E0
:10131000EF00D036832701006392070683278102FE
:1013200083A787031387F7FF8327810223ACE70294
:101330008327810283A70700639A0700EF30C076F6
:10134000130705008327810223A2E7008327810278
:1013500083A70701638E0704832781029387070110
:1013600013850700EF20C07C1307050093071000CA
:101370006310F704EFF0CFA16F0080038327810291
:101380000327410223A6E7008327810283A74702A0
:101390006380070283278102938747021385070032
:1013A000EF2000799307050063840700EFF04F9E5C
:1013B000EF30C064930710006F00000C83274100DA
:1013C00063980700EF308063930700006F00C00A46
:1013D0008327C102639C07009307C101138507009F
:1013E000EF20101A930710002326F102EF3000615E
:1013F000EF30C05C130741009307C101930507005C
:1014000013850700EF20901C93070500639C0704D9
:1014100003258102EF00103E93070500638A07044D
:101420008327810283A70700639E0700EF300059DE
:101430008327810283A7470013850700EF30802EA2
:10144000EF30C05B83278102938747020327410067
:101450009305070013850700EF200048EFF04F9336
:101460006F000001EF308059930700006F00C0004B
:10147000EF30C0586FF09FE7138507008320C1034A
:101480001301010467800000130101FD23261102EE
:101490002326A1002324B1002322C1002320D10050
:1014A0008327C100232CF100832781016396070065
:1014B000737004306F000000832781006398070079
:1014C0008327810183A70704639607009307100011
:1014D0006F0080009307000063960700737004306C
:1014E0006F0000000327010093072000631AF70034
:1014F0008327810103A7C703930710006316F70032
:10150000930710006F0080009307000063960700A8
:10151000737004306F000000EFF0CF9E930705005A
:10152000232AF1008327810103A7870383278101F1
:1015300083A7C7036368F700032701009307200010
:101540006310F7080326010083258100032581012C
:10155000EF00807A8327810103A787049307F0FFB8
:101560006310F7048327810183A74702638407047C
:10157000832781019387470213850700EF20405B93
:1015800093070500638807028327410063840702ED
:10159000832741001307100023A0E7006F0080019C
:1015A0008327810183A7870413871700832781017D
:1015B00023A4E70493071000232EF1006F0080009E
:1015C000232E01008327410113850700EFF0CF91FF
:1015D0008327C101138507008320C1021301010382
:1015E00067800000130101FD232611022326A100BC
:1015F0002324B1008327C100232CF100832781011C
:1016000063960700737004306F0000008327810128
:1016100083A7070463860700737004306F0000001F
:101620008327810183A7070063980700832781012F
:1016300083A7470063960700930710006F008000A0
:101640009307000063960700737004306F0000007A
:10165000EFF04F8B93070500232AF10083278101C8
:1016600003A787038327810183A7C7036372F70852
:101670008327810183A787031387170083278101AD
:1016800023ACE7028327810103A787049307F0FFB8
:101690006310F7048327810183A74702638407044B
:1016A000832781019387470213850700EF20404875
:1016B000930705006388070283278100638407027C
:1016C000832781001307100023A0E7006F0080012B
:1016D0008327810183A7870413871700832781014C
:1016E00023A4E70493071000232EF1006F0080006D
:1016F000232E01008327410113850700EFE0DFFE61
:101700008327C101138507008320C1021301010350
:1017100067800000130101FC232E11022326A10083
:101720002324B1002322C1002320D100232601025B
:101730008327C1002324F1028327810263960700D7
:10174000737004306F0000008327810063980700E6
:101750008327810283A7070463960700930710007D
:101760006F008000930700006396070073700430D9
:101770006F000000EF2010769307050063960700C6
:101780008327410063960700930710006F008000D5
:101790009307000063960700737004306F00000029
:1017A000EF30C0218327810283A787036382070C60
:1017B0008327810283A7C7002322F10283258100AA
:1017C00003258102EF00806B8327010063920706E7
:1017D0008327810283A787031387F7FF832781026B
:1017E00023ACE7028327810283A70700639A0700DF
:1017F000EF30802B130705008327810223A2E70027
:101800008327810283A70701638E07048327810250
:101810009387070113850700EF2080311307050028
:10182000930710006310F704EFE09FD66F0080036A
:10183000832781020327410223A6E7008327810231
:1018400083A74702638007028327810293874702A9
:1018500013850700EF20C02D930705006384070060
:10186000EFE01FD3EF308019930710006F00801155
:101870008327410063980700EF304018930700006A
:101880006F0040108327C102639C07009307C101CA
:1018900013850700EF20C04E930710002326F102A6
:1018A000EF30C015EF10407BEF30401183278102ED
:1018B00003A747049307F0FF6316F700832781020D
:1018C00023A207048327810203A787049307F0FF5D
:1018D0006316F7008327810223A40704EF30001268
:1018E000130741009307C101930507001385070003
:1018F000EF20C04D93070500639E07060325810274
:10190000EF00406F93070500638E07048327810271
:1019100083A70700639E0700EF30400A83278102F8
:1019200083A7470013850700EF20D05FEF30000D3D
:10193000832781029387470203274100930507000D
:1019400013850700EF10507903258102EF00C05B7B
:10195000EF10C07293070500E39407E4EFE05FC364
:101960006FF01FE403258102EF00005AEF100071B1
:101970006FF01FE303258102EF000059EF100070A4
:1019800093070000138507008320C103130101049E
:1019900067800000130101FD232611022326A10008
:1019A0002324B1002322C1008327C100232CF1008E
:1019B0008327810163960700737004306F00000075
:1019C00083278100639807008327810183A7070489
:1019D00063960700930710006F00800093070000D4
:1019E00063960700737004306F000000EFE09FD132
:1019F00093070500232AF1008327810183A787032A
:101A0000638807088325810003258101EF000047D3
:101A10008327810183A787031387F7FF832781012A
:101A200023ACE7028327810103A747049307F0FF54
:101A30006310F7048327810183A7070163840704E8
:101A4000832781019387070113850700EF20400E4C
:101A50009307050063880702832741006384070218
:101A6000832741001307100023A0E7006F008001C7
:101A70008327810183A747041387170083278101E8
:101A800023A2E70493071000232EF1006F008000CB
:101A9000232E01008327410113850700EFE0DFC4F7
:101AA0008327C101138507008320C10213010103AD
:101AB00067800000130101FD232611022326A100E7
:101AC0002324B1008327C100232CF1008327810147
:101AD00063960700737004306F0000008327810055
:101AE000639807008327810183A707046396070093
:101AF000930710006F0080009307000063960700B3
:101B0000737004306F0000008327810183A70704EE
:101B100063960700737004306F000000EFE09FBE13
:101B200093070500232AF1008327810183A78703F8
:101B3000638A07028327810183A7C7002328F10056
:101B40008325810003258101EF0040338327810134
:101B50000327010123A6E70093071000232EF100BD
:101B60006F008000232E01008327410113850700A9
:101B7000EFE09FB78327C101138507008320C102CF
:101B80001301010367800000130101FD23261102E8
:101B90002326A1008327C1006396070073700430D9
:101BA0006F000000EF2090618327C10083A78703A7
:101BB000232EF100EF2090648327C10113850700D5
:101BC0008320C1021301010367800000130101FD9E
:101BD000232611022326A1008327C100232EF10012
:101BE0008327C10163960700737004306F00000003
:101BF000EF20D05C8327C10103A7C7038327C1015E
:101C000083A78703B307F740232CF100EF20105F71
:101C100083278101138507008320C102130101037B
:101C200067800000130101FE2326A1008327C10065
:101C300063960700737004306F0000008327C100B3
:101C400083A78703232EF1008327C1011385070093
:101C50001301010267800000130101FD2326110218
:101C60002326A1008327C100232EF1008327C10171
:101C700063960700737004306F0000000325C101F4
:101C8000EF0040520325C101EF4050371300000020
:101C90008320C1021301010367800000130101FFCB
:101CA0002326A1008327C10083A7C704138507004B
:101CB0001301010167800000130101FF2326A10029
:101CC0002324B1008327C1000327810023A6E70452
:101CD000130000001301010167800000130101FFE0
:101CE0002326A1008327C10083C7070513850700AA
:101CF0001301010167800000130101FD2326110279
:101D00002326A1002324B1002322C100232E010099
:101D10008327C10083A70704639807028327C100B4
:101D200083A70700639807128327C10083A7470092
:101D300013850700EF20D034232EA1008327C10094
:101D400023A207006F000011832741006394070658
:101D50008327C10003A787008327C10083A7070447
:101D6000138607008325810013050700EF40D03F4D
:101D70008327C10003A787008327C10083A7070427
:101D80003307F7008327C10023A4E7008327C1009E
:101D900003A787008327C10083A74700636CF70A66
:101DA0008327C10003A707008327C10023A4E700FE
:101DB0006F00400A8327C10003A7C7008327C10023
:101DC00083A70704138607008325810013050700F6
:101DD000EF4090398327C10003A7C7008327C100C4
:101DE00083A70704B307F0403307F7008327C10038
:101DF00023A6E7008327C10003A7C7008327C100EC
:101E000083A707006372F7028327C10003A7470077
:101E10008327C10083A70704B307F0403307F70007
:101E20008327C10023A6E700032741009307200072
:101E30006312F7028327C10083A78703638C07001F
:101E40008327C10083A787031387F7FF8327C10078
:101E500023ACE7028327C10083A7870313871700FA
:101E60008327C10023ACE7028327C1011385070044
:101E70008320C1021301010367800000130101FEEA
:101E8000232E11002326A1002324B1008327C100A3
:101E900083A70704638207068327C10003A7C7003F
:101EA0008327C10083A707043307F7008327C100F6
:101EB00023A6E7008327C10003A7C7008327C1002B
:101EC00083A74700636AF7008327C10003A70700C1
:101ED0008327C10023A6E7008327C10003A7C7000B
:101EE0008327C10083A70704138607009305070013
:101EF00003258100EF405027130000008320C1011B
:101F00001301010267800000130101FE232E11005E
:101F10002326A100EF20902A6F0000048327C10030
:101F200083A74702638207048327C1009387470280
:101F300013850700EF10D03F930705006384070067
:101F4000EF10D0788327C10083A787041387F7FF9A
:101F50008327C10023A4E7048327C10083A7870444
:101F6000E34EF0FA6F008000130000008327C100E9
:101F70001307F0FF23A4E704EF205028EF201024DC
:101F80006F0000048327C10083A707016382070451
:101F90008327C1009387070113850700EF1050398D
:101FA0009307050063840700EF1050728327C10078
:101FB00083A747041387F7FF8327C10023A2E70401
:101FC0008327C10083A74704E34EF0FA6F00800027
:101FD000130000008327C1001307F0FF23A2E704CA
:101FE000EF20D021130000008320C1011301010262
:101FF00067800000130101FD232611022326A100A2
:10200000EF20D01B8327C10083A7870363980700B5
:1020100093071000232EF1006F008000232E010093
:10202000EF20D01D8327C101138507008320C10243
:102030001301010367800000130101FE2326A100A4
:102040008327C10063960700737004306F0000009F
:102050008327C10083A787036398070093071000B5
:10206000232EF1006F008000232E01008327C10181
:10207000138507001301010267800000130101FDB1
:10208000232611022326A100EF2050138327C1002D
:1020900003A787038327C10083A7C7036318F7003B
:1020A00093071000232EF1006F008000232E010003
:1020B000EF20D0148327C101138507008320C102BC
:1020C0001301010367800000130101FE2326A10014
:1020D0008327C10063960700737004306F0000000F
:1020E0008327C10003A787038327C10083A7C703F2
:1020F0006318F70093071000232EF1006F00800093
:10210000232E01008327C10113850700130101025B
:1021100067800000130101FE2326A1002324B100E3
:10212000232E01006F008006177703001307875BDB
:102130008327C10193973700B307F70083A70700F0
:1021400063900704177703001307C7598327C1015A
:1021500093973700B307F7000327810023A0E70018
:1021600017770300130707588327C1019397370098
:10217000B307F7000327C10023A2E7006F00C001E7
:102180008327C10193871700232EF1000327C10184
:1021900093077000E3FAE7F813000000130101024F
:1021A00067800000130101FE2326A100232E0100F9
:1021B0006F00C004177703001307C7528327C101BC
:1021C00093973700B307F70083A747000327C100A1
:1021D0006310F702177703001307C7508327C10165
:1021E00093973700B307F70023A007006F00C001E3
:1021F0008327C10193871700232EF1000327C10114
:1022000093077000E3F8E7FA1300000013010102DE
:1022100067800000130101FD232611022326A1007F
:102220002324B1002322C1008327C100232EF10003
:10223000EF20C0788327C10103A747049307F0FF6D
:102240006316F7008327C10123A207048327C10176
:1022500003A787049307F0FF6316F7008327C101E4
:1022600023A40704EF2080798327C10183A7870374
:10227000639E07008327C10193874702032641001D
:102280008325810013850700EF10007F0325C1011E
:10229000EFF09FC7130000008320C1021301010368
:1022A00067800000130101FC232E1102232EA100E0
:1022B000232CB1002328D1002326E1002324F100A0
:1022C000232201012320110193070600231BF100A3
:1022D0008327C10163960700737004306F0000000C
:1022E0000327C1009307900063F6E7007370043082
:1022F0006F000000835761018325410013850700AB
:10230000EF10D07E2324A102832781026386071C5D
:102310008327810203A7070383566101B7070040A3
:102320009387F7FFB387F60093972700B307F7006B
:102330002322F1028327410293F7C7FF2322F102F0
:102340008327410293F737006386070073700430D8
:102350006F00000083576101138707008326010087
:102360000326C1008325810103258102EF1050411E
:10237000032601018325C10103254102EFE08FBA45
:10238000130705008327810223A0E700832781002C
:1023900063880700832781000327810223A0E700C9
:1023A000EF20C06197E701009387072183A707000B
:1023B0001387170097E701009387072023A0E70002
:1023C00097E701009387070283A707006398070236
:1023D00097E70100938707010327810223A0E70005
:1023E00097E701009387471D03A707009307100095
:1023F0006312F704EF10904B6F00C00397E70100E2
:102400009387471C83A707006396070297E701009D
:10241000938747FD83A7070083A7C7020327C1004F
:10242000636AF70097E701009387C7FB03278102E0
:1024300023A0E70097E701009387C71983A7070048
:102440001387170097E701009387C71823A0E700B9
:1024500097E701009387071803A7070083278102E6
:1024600023A4E7048327810203A7C70297E701009B
:102470009387071583A7070063FCE7008327810282
:1024800003A7C70297E701009387871323A0E700FC
:102490008327810203A7C7029307070093972700AA
:1024A000B387E7009397270017E70100130747FD5D
:1024B0003387E700832781029387470093850700CE
:1024C00013050700EFE08FB8930710002326F102F1
:1024D000EF20C0526F00C0009307F0FF2326F102E7
:1024E0000327C102930710006318F70297E7010062
:1024F0009387470D83A707006380070297E70100D2
:10250000938747EE83A7070083A7C7020327C1006D
:1025100063F4E700EFE0CF878327C102138507004C
:102520008320C1031301010467800000130101FD32
:10253000232611022326A100EF2040488327C10053
:10254000639A070097E701009387C7E983A707000D
:102550006F0080008327C100232EF1008327C10173
:102560009387470013850700EFE08FC28327C101DF
:1025700083A78702638A07008327C10193878701A6
:1025800013850700EFE0CFC08327C1019387470081
:102590009385070017E50100130545FFEFE00FAB3A
:1025A00097E701009387C7FF83A7070013871700EA
:1025B00097E701009387C7FE23A0E70097E7010094
:1025C0009387470183A707001387170097E7010048
:1025D0009387470023A0E700EF20404297E70100E0
:1025E000938747FE83A707006382070497E70100EC
:1025F000938747DF83A707000327C1016312F70210
:1026000097E70100938787FD83A70700638607008C
:10261000737004306F000000EFD09FF76F0000016F
:10262000EF20C039EF208001EF20403D1300000073
:102630008320C1021301010367800000130101FD23
:10264000232611022326A1002324B100232E0100FA
:102650008327C10063960700737004306F00000089
:102660008327810063960700737004306F000000B9
:1026700097E70100938787F683A707006386070023
:10268000737004306F000000EF00101D97E7010029
:102690009387C7F283A70700232CF1008327C1008B
:1026A00083A7070003278100B307F700232AF1005F
:1026B0008327C10083A70700032781016376F70200
:1026C0008327C10083A70700032741016370F70434
:1026D000032741018327810163FAE7029307100072
:1026E000232EF1006F0080028327C10083A707001B
:1026F000032741016368F700032741018327810114
:1027000063F6E70093071000232EF1008327C10032
:102710000327410123A0E7008327C1016382070249
:1027200097E70100938707CC83A7070093874700AB
:1027300013850700EFE0CFA503254101EF10502FCF
:10274000EF00D0132328A100832701016394070021
:10275000EFD01FE4130000008320C1021301010326
:1027600067800000130101FD232611022326A1002A
:10277000232E01008327C1006380070697E701002D
:102780009387C7E583A7070063860700737004304B
:102790006F000000EF00500C97E70100938707E2FD
:1027A00083A707000327C100B307F700232CF1001C
:1027B00097E70100938707C383A707009387470024
:1027C00013850700EFE0CF9C03258101EF10502611
:1027D000EF00D00A232EA1008327C10163940700D4
:1027E000EFD01FDB130000008320C102130101039F
:1027F00067800000130101FD232611022326A1009A
:102800008327C100232CF1008327810163960700F1
:10281000737004306F00000097E70100938787BC56
:1028200083A70700032781016316F700232E010009
:102830006F00400AEF2080188327810183A747019A
:10284000232AF100EF20801B97E70100938747D2EE
:1028500083A7070003274101630CF70097E70100F6
:10286000938747D183A70700032741016318F70027
:1028700093072000232EF1006F00C00503274101BC
:1028800097E70100938707D26314F702832781013A
:1028900083A787026398070093073000232EF10077
:1028A0006F00400393072000232EF1006F00800289
:1028B0000327410197E70100938747CD6318F7008D
:1028C00093074000232EF1006F00C0009307100013
:1028D000232EF1008327C101138507008320C10245
:1028E0001301010367800000130101FD232611027B
:1028F0002326A100EF20800C8327C100639A0700E4
:1029000097E70100938707AE83A707006F00800059
:102910008327C100232EF1008327C10183A7C702AB
:10292000232CF100EF20800D832781011385070000
:102930008320C1021301010367800000130101FD20
:10294000232611022326A100EFD0DFDB9307050029
:10295000232EF1008327C100639A070097E7010047
:10296000938747A883A707006F0080008327C100D3
:10297000232CF1008327810183A7C702232AF100BA
:102980008327C10113850700EFD01FD6832741019C
:10299000138507008320C102130101036780000033
:1029A000130101FD232611022326A1002324B100D7
:1029B000232E0100032781009307900063F6E700B0
:1029C000737004306F0000000327810093079000AC
:1029D00063F6E700930790002324F100EF10107EC8
:1029E0008327C100639A070097E701009387879FB9
:1029F00083A707006F0080008327C100232CF1000C
:102A00008327810183A70705232AF10003274101BA
:102A100083278100630EF716032781008327410176
:102A200063FEE70297E701009387C79B83A7070030
:102A3000032781016302F70497E701009387879AD0
:102A400083A7070083A7C702032781006366F702F5
:102A500093071000232EF1006F00000297E701009A
:102A60009387479883A70700032781016316F70020
:102A700093071000232EF1008327810183A7C7024B
:102A80002328F1008327810103A7070583278101FC
:102A900083A7C7026318F7008327810103278100FA
:102AA00023A6E702832781010327810023A8E704E7
:102AB0008327810183A7870163CC07001307A00048
:102AC000832781003307F7408327810123ACE70088
:102AD0008327810183A6470103270101930707008C
:102AE00093972700B387E7009397270017E7010024
:102AF00013070799B387E7006396F6009307100062
:102B00006F00800093070000638C07068327810114
:102B10009387470013850700EFD09FE78327810144
:102B200003A7C70297E70100938787A983A7070038
:102B300063FCE7008327810103A7C70297E7010031
:102B4000938707A823A0E7008327810103A7C70273
:102B50009307070093972700B387E7009397270011
:102B600017E701001307C7913387E7008327810127
:102B7000938747009385070013050700EFD01FCD0B
:102B80000327C101930710006314F700EFD05FA083
:102B9000EF10D066130000008320C102130101036F
:102BA00067800000130101FD232611022326A100E6
:102BB000EF10D0608327C100639A070097E70100F8
:102BC0009387478283A707006F0080008327C10097
:102BD000232EF1008327C101938747001385070047
:102BE000EFD01FDB8327C10183A78702638A070019
:102BF0008327C1019387870113850700EFD05FD931
:102C00008327C101938747009385070017E50100DB
:102C100013054599EFD09FC3EF10505E97D7010081
:102C20009387477C83A707000327C1016314F70636
:102C300097E701009387079983A70700638207023C
:102C400097E701009387879983A7070063860700AA
:102C5000737004306F000000EFD09F936F00400549
:102C600097E701009387079403A7070097E7010000
:102C70009387879483A70700631AF70097D701000B
:102C80009387477623A007006F008002EF0090280B
:102C90006F00000297E701009387C79283A70700A0
:102CA00063880700EF109051EF105019EF10105586
:102CB000130000008320C10213010103678000009C
:102CC000130101FE2326A100232E01008327C1004A
:102CD000232CF1008327C100639607007370043032
:102CE0006F0000008327810103A7470197E70100D8
:102CF0009387478B6316F700930710006F008000DF
:102D000093070000638E07028327810103A78702D0
:102D100097E70100938747866304F70283278101C1
:102D200083A7870263960700930710006F00800057
:102D3000930700006386070093071000232EF1001D
:102D40008327C1011385070013010102678000007A
:102D5000130101FD232611022326A1008327C100B0
:102D6000232EF1008327C10063960700737004309F
:102D70006F0000008327C1016384070C97D701000F
:102D80009387476683A707000327C101630AF70AF1
:102D9000EF10D0420325C101EFF09FF213070500A9
:102DA00093071000631CF7088327C101938747002E
:102DB00013850700EFD0DFBD8327C10103A7C7023A
:102DC00097D701009387C77F83A7070063FCE700BD
:102DD0008327C10103A7C70297D701009387477EC6
:102DE00023A0E7008327C10103A7C70293070700B9
:102DF00093972700B387E7009397270017D7010021
:102E0000130707683387E7008327C10193874700CB
:102E10009385070013050700EFD05FA38327C10147
:102E200003A7C70297D701009387C75B83A7070053
:102E300083A7C7026364F700EFD08FF5EF10103C53
:102E4000130000008320C10213010103678000000A
:102E5000130101FD232611022326A100232E0100C8
:102E60008327C100232CF1008327C100639607004C
:102E7000737004306F000000EFD0DF889307050007
:102E8000232AF10003258101EFF09FE313070500DA
:102E9000930710006314F70C97D70100938707740A
:102EA00083A707006390070A8327810103A7C7024E
:102EB00097D701009387075383A7070083A7C7020B
:102EC0006366F70093071000232EF100832781012A
:102ED0009387470013850700EFD09FAB83278101BD
:102EE00003A7C70297D701009387876D83A70700C1
:102EF00063FCE7008327810103A7C70297D701007E
:102F00009387076C23A0E7008327810103A7C702EB
:102F10009307070093972700B387E700939727004D
:102F200017D701001307C7553387E70083278101AF
:102F3000938747009385070013050700EFD01F9183
:102F40006F00C00183278101938787019385070064
:102F500017D5010013054562EFD05F8F832741012C
:102F600013850700EFD04FF88327C10113850700B1
:102F70008320C1021301010367800000130101FED9
:102F8000232E11009308000013080000930700008F
:102F900013070000930600001306004097D50100B8
:102FA0009385450617150000130505FBEFF08FAF5D
:102FB0002326A1000327C100930710006316F70022
:102FC000EF20C03A2326A1000327C1009307100079
:102FD000631EF7027370043097D701009387C75FB1
:102FE0001307F0FF23A0E70097D701009387875DC1
:102FF0001307100023A0E70097D701009387075C11
:1030000023A00700EFD00FBE6F0040018327C1004F
:1030100063960700737004306F0000001300000017
:103020008320C1011301010267800000130101FF29
:10303000232611007370043097D7010093878758B7
:1030400023A00700EFD04FCC130000008320C10065
:10305000130101016780000097D70100938707588B
:1030600083A707001387170097D701009387075797
:1030700023A0E7001300000067800000130101FE99
:10308000232E11002326010097D7010093870755AF
:1030900083A7070063960700737004306F00000079
:1030A000EF10D01197D701009387475383A70700EC
:1030B0001387F7FF97D701009387475223A0E700B4
:1030C00097D701009387875183A70700639407165A
:1030D00097D701009387474E83A70700638C071497
:1030E0006F00800C97D701009387074983A7C7001B
:1030F00083A7C7002324F1008327810093878701DA
:1031000013850700EFD0DF8883278100938747006E
:1031100013850700EFD0DF878327810003A7C7024D
:1031200097D701009387C74983A7070063FCE7008F
:103130008327810003A7C70297D7010093874748D9
:1031400023A0E7008327810003A7C7029307070096
:1031500093972700B387E7009397270017D70100BD
:10316000130707323387E7008327810093874700DF
:103170009385070013050700EFD04FED83278100EB
:1031800003A7C70297D701009387C72583A7070026
:1031900083A7C702636AF70097D7010093870743A5
:1031A0001307100023A0E70097D701009387C73CBF
:1031B00083A70700E39807F297D701009387C740DA
:1031C00083A70700638807046F00C003EF00002B8C
:1031D00093070500638A070097D701009387073F8D
:1031E0001307100023A0E70097D701009387C73D7E
:1031F00083A707001387F7FF97D701009387C73C82
:1032000023A0E70097D701009387073C83A7070017
:10321000E39E07FA97D701009387473B03A7070070
:10322000930710006318F700930710002326F1009E
:10323000EFD00FB6EF10807C8327C1001385070005
:103240008320C1011301010267800000130101FE08
:10325000232E1100EF10807697D701009387073651
:1032600083A707002326F100EF1040798327C100D0
:10327000138507008320C10113010102678000004C
:10328000130101FE232E1100EFD0CFC793070500D5
:103290002326F10097D701009387473283A70700C1
:1032A0002324F1008327C10013850700EFD0CFC38B
:1032B00083278100138507008320C10113010102C8
:1032C0006780000097D701009387072F83A7070027
:1032D0001385070067800000130101FD23261102FA
:1032E0002326A1002324B1002322C100232E0100A4
:1032F0009307A000232CF100EFF01FD697D7010011
:103300009387872B83A7070003278100636CF7143B
:10331000832781019387F7FF232CF1008327C101C5
:10332000939757000327C100B306F70003278101D5
:103330009307070093972700B387E7009397270029
:1033400017D701001307C713B387E7001306100050
:103350009385070013850600EF108004130705000E
:103360008327C101B387E700232EF1008327810162
:10337000E39007FA8327C101939757000327C10001
:103380003307F70097D701009387871E83A70700AD
:10339000130620009385070013050700EF10400077
:1033A000130705008327C101B387E700232EF1002F
:1033B0008327C101939757000327C1003307F70004
:1033C00097D701009387071B83A7070013062000E8
:1033D0009385070013050700EF00907C1307050095
:1033E0008327C101B387E700232EF1008327C101A2
:1033F000939757000327C100B307F7001306400057
:1034000097D501009385851813850700EF00507943
:10341000130705008327C101B387E700232EF100BE
:103420008327C101939757000327C100B307F70013
:103430001306300097D501009385C5161385070044
:10344000EF001076130705008327C101B387E7005B
:10345000232EF10083274100638607008327410064
:1034600023A00700EFF09FC18327C1011385070048
:103470008320C1021301010367800000130101FDD5
:1034800023261102232E010097D7010093870715E9
:1034900083A70700639C072297D701009387071231
:1034A00083A707001387170097D701009387071199
:1034B00023A0E70097D701009387471083A7070051
:1034C000232CF10083278101639C070697D7010015
:1034D0009387070A83A7070083A70700638607006F
:1034E000737004306F00000097D70100938747087E
:1034F00083A70700232AF10097D701009387870746
:1035000003A7070097D701009387870623A0E7004A
:1035100097D70100938707060327410123A0E700FF
:1035200097D701009387C70A83A70700138717005F
:1035300097D701009387C70923A0E700EF10001079
:1035400097D701009387470983A7070003278101C5
:10355000636CF71297D701009387870183A7070051
:1035600083A7070063960700930710006F00800091
:1035700093070000638C070097D701009387C70566
:103580001307F0FF23A0E7006F00001097D701009A
:10359000938707FE83A7070083A7C70083A7C700F9
:1035A0002328F1008327010183A747002326F10088
:1035B000032781018327C100637CF70097D70100AF
:1035C000938787010327C10023A0E7006F00C00B8A
:1035D000832701019387470013850700EFD04FBB76
:1035E0008327010183A78702638A070083270101DC
:1035F0009387870113850700EFD08FB983270101D7
:1036000003A7C70297D70100938787FB83A707000B
:1036100063FCE7008327010103A7C70297D70100D6
:10362000938707FA23A0E7008327010103A7C702B6
:103630009307070093972700B387E7009397270026
:1036400017D701001307C7E33387E700832701017A
:10365000938747009385070013050700EFD00F9F5E
:103660008327010103A7C70297D70100938787D754
:1036700083A7070083A7C702E36EF7EC9307100048
:10368000232EF1006FF01FED97D70100938787D5A8
:1036900083A7070003A7C70297D60100938646DEDB
:1036A0009307070093972700B387E70093972700B6
:1036B000B387F60003A707009307100063F6E7023D
:1036C00093071000232EF1006F00000297D701002E
:1036D000938787EF83A707001387170097D7010009
:1036E000938787EE23A0E70097D70100938707EE23
:1036F00083A707006386070093071000232EF100BD
:103700008327C101138507008320C1021301010330
:1037100067800000130101FE232E110097D70100DE
:103720009387C7EB83A70700638C070097D7010037
:103730009387C7E91307100023A0E7006F00C018A4
:1037400097D70100938787E823A0070097D7010048
:10375000938747C983A7070083A707032326F100A0
:10376000B7A7A5A59387575A2324F1008327C10043
:1037700083A70700032781006310F7048327C10094
:103780009387470083A70700032781006316F7028A
:103790008327C1009387870083A707000327810041
:1037A000631CF7008327C1009387C70083A7070026
:1037B000032781006302F70697D70100938787C22A
:1037C00003A7070097D701009387C7C183A7070006
:1037D000938747039385070013050700EF404019BF
:1037E0006F00800397D70100938787DD83A70700C9
:1037F00063960700737004306F00000097D70100D4
:10380000938707DC83A707001387F7FF97D701008B
:10381000938707DB23A0E70097D70100938747DA58
:1038200003A7070097D60100938686C59307070074
:1038300093972700B387E70093972700B387F60095
:1038400083A70700E38007FA97D70100938747D73C
:1038500003A707009307070093972700B387E700A4
:103860009397270017D70100130787C1B387E70095
:103870002322F1008327410083A7470003A74700C5
:103880008327410023A2E7008327410003A74700C5
:103890008327410093878700631CF700832741003B
:1038A00083A7470003A747008327410023A2E7001F
:1038B0008327410083A7470003A7C70097D70100CC
:1038C000938747B223A0E700130000008320C101C3
:1038D0001301010267800000130101FD232611027C
:1038E0002326A1002324B1008327C100639607008B
:1038F000737004306F00000097D70100938787AE84
:1039000083A7070093878701938507000325C100DC
:10391000EFC09FFB97D701009387C7AC83A7070031
:103920009387470013850700EFD08F860327810018
:103930009307F0FF6314F70297D70100938787AAD4
:1039400083A70700938747009385070017D50100D9
:10395000130545C5EFC09FEF6F00400297D70100E8
:103960009387C7C583A7070003278100B307F70024
:10397000232EF1000325C101EF00900B130000007E
:103980008320C1021301010367800000130101FDC0
:10399000232611022326A1002324B1002322C100E3
:1039A0008327C10063960700737004306F00000026
:1039B00097D70100938787C283A707006396070004
:1039C000737004306F00000097D70100938787A1C0
:1039D00083A70700832681003707008033E7E600CE
:1039E00023ACE70097D701009387C79F83A7070001
:1039F00093878701938507000325C100EFC01FE56A
:103A000097D701009387079E83A7070093874700F6
:103A100013850700EFC0DFF7032741009307F0FF8E
:103A20006314F70297D701009387C79B83A707000A
:103A3000938747009385070017D50100130585B6C6
:103A4000EFC0DFE06F00400297D70100938707B710
:103A500083A7070003274100B307F700232EF100D7
:103A60000325C101EF00C07C130000008320C102C8
:103A70001301010367800000130101FD23261102D9
:103A80002326A1002324B1002322C1008327C100E3
:103A900063960700737004306F00000097D7010031
:103AA0009387479483A7070093878701938507002F
:103AB0000325C100EFC09FD997D701009387879254
:103AC00083A707009387470013850700EFC05FECCB
:103AD00003274100930710006314F70297D70100F2
:103AE0009387479083A70700938747009385070034
:103AF00017D50100130505ABEFC05FD56F0040027D
:103B000097D70100938787AB83A70700032781001E
:103B1000B307F700232EF1000325C101EF00407128
:103B2000130000008320C10213010103678000001D
:103B3000130101FD232611022326A1008327C100C2
:103B400083A7C70083A7C700232CF1008327810127
:103B500063960700737004306F00000083278101B3
:103B60009387870113850700EFC09FE297D7010075
:103B70009387C7A683A70700639E07068327810153
:103B80009387470013850700EFC09FE083278101DB
:103B900003A7C70297D70100938787A283A70700CF
:103BA00063FCE7008327810103A7C70297D70100C1
:103BB000938707A123A0E7008327810103A7C702FA
:103BC0009307070093972700B387E7009397270091
:103BD00017D701001307C78A3387E70083278101BE
:103BE000938747009385070013050700EFC01FC6A2
:103BF0006F00C001832781019387870193850700A8
:103C000017D5010013054597EFC05FC483278101D5
:103C100003A7C70297C701009387C77C83A7070044
:103C200083A7C70263F0E70293071000232EF10079
:103C300097D70100938787991307100023A0E70007
:103C40006F008000232E01008327C1011385070028
:103C50008320C1021301010367800000130101FDED
:103C6000232611022326A1002324B10097D70100A7
:103C70009387C79683A70700639607007370043085
:103C80006F00000003278100B70700803367F7004B
:103C90008327C10023A0E7008327C10083A7C700B3
:103CA000232CF10083278101639607007370043091
:103CB0006F0000000325C100EFC09FCD8327810165
:103CC0009387470013850700EFC09FCC83278101AE
:103CD00003A7C70297D701009387878E83A70700A2
:103CE00063FCE7008327810103A7C70297D7010080
:103CF0009387078D23A0E7008327810103A7C702CD
:103D00009307070093972700B387E700939727004F
:103D100017C701001307C7763387E70083278101A0
:103D2000938747009385070013050700EFC01FB274
:103D30008327810103A7C70297C701009387876A7A
:103D400083A7070083A7C70263F0E7029307100069
:103D5000232EF10097D701009387478713071000A0
:103D600023A0E7006F008000232E01008327C101FC
:103D7000138507008320C10213010103678000003F
:103D8000130101FF2326A1008327C10063960700CA
:103D9000737004306F00000097D70100938747834A
:103DA00003A707008327C10023A0E70097D70100DE
:103DB0009387C78003A707008327C10023A2E700DA
:103DC000130000001301010167800000130101FDD1
:103DD000232611022326A1002324B1008327C1003A
:103DE00063960700737004306F0000008327810022
:103DF00063960700737004306F000000EF00103C02
:103E000097C701009387877B83A70700232CF100C6
:103E10008327810003A707009307F0FF6316F700CD
:103E2000232E01006F0000098327C10003A70700AC
:103E300097C701009387C77983A707006300F7023C
:103E40008327C10083A74700032781016368F70028
:103E500093071000232EF1006F00C0058327C100D7
:103E600083A74700032781013307F7408327810099
:103E700083A70700637CF7028327810003A707005D
:103E80008327C10083A6470083278101B387F640BB
:103E90003307F7008327810023A0E7000325C10033
:103EA000EFF01FEE232E01006F00C00093071000FB
:103EB000232EF100EF0090348327C1011385070002
:103EC0008320C102130101036780000097C701002E
:103ED0009387C76F1307100023A0E70013000000AB
:103EE00067800000130101FE2326A1008327C10083
:103EF000638E07008327C100232CF10083278101F3
:103F000083A7C704232EF1006F008000232E010039
:103F10008327C10113850700130101026780000098
:103F2000130101FE2326A1002324B1008327C10031
:103F3000638C07008327C100232EF1008327C10172
:103F40000327810023A6E7041300000013010102E8
:103F500067800000130101FE232E11002326A1001B
:103F6000EF00002197C701009387875103A707003F
:103F700093071000E3F6E7FEEFC08FE16FF05FFEFE
:103F8000130101FC232E1102232EA100232CB100CA
:103F9000232AC1002328D100930707002317F1002B
:103FA000232601026F004004032781018327C102F9
:103FB000B307F70003C707008326C1018327C102A7
:103FC000B387F600238AE702032781018327C10212
:103FD000B307F70083C70700638007028327C10286
:103FE000938717002326F1020327C1029307F000ED
:103FF000E3FCE7FA6F008000130000008327C10193
:10400000A3810704032741019307900063F6E700AB
:1040100093079000232AF1008327C1010327410160
:1040200023A6E7028327C1010327410123A8E70450
:104030008327C10123AA07048327C101938747006F
:1040400013850700EFC0CFFE8327C1019387870147
:1040500013850700EFC0CFFD8327C1010327C101EE
:1040600023A8E7001307A000832741013307F74087
:104070008327C10123ACE7008327C1010327C101C6
:1040800023A2E7028327C10123A207048327C101DA
:1040900023AC07048327C10123AE070413000000EB
:1040A0008320C1031301010467800000130101FE96
:1040B000232E1100232601006F0080030327C10077
:1040C0009307070093972700B387E700939727008C
:1040D00017C701001307C73AB387E7001385070026
:1040E000EFC08FEF8327C100938717002326F100CD
:1040F0000327C10093079000E3F2E7FC17C5010016
:1041000013058544EFC04FED17C5010013050545A4
:10411000EFC08FEC17C5010013050546EFC0CFEBCC
:1041200017C5010013058546EFC00FEB17C5010049
:1041300013054547EFC04FEA97C7010093874743F0
:1041400017C701001307474023A0E70097C70100E6
:104150009387474217C701001307474023A0E70092
:10416000130000008320C1011301010267800000D9
:10417000130101FE232E11006F008009EFE0DFED37
:1041800097C701009387874083A7070093B717005D
:1041900093F7F70F2326F100EFE05FEE8327C100CE
:1041A00063980706EF00900197C701009387073EC9
:1041B00083A7C70083A7C7002324F10083278100BA
:1041C0009387470013850700EFC08FFC97C7010056
:1041D0009387873E83A707001387F7FF97C70100E0
:1041E0009387873D23A0E70097C701009387473B4C
:1041F00083A707001387F7FF97C701009387473A04
:1042000023A0E700EF00807F03258100EF00C03F7F
:1042100097C701009387C73883A70700E39007F685
:10422000130000008320C101130101026780000018
:10423000130101FE232E11002326A10097C70100C0
:104240009387471A83A707000327C10023A2E7002B
:1042500097C701009387873683A707000327C1000C
:104260006378F70297C701009387C73003A7070059
:1042700097C701009387071783A707009387470015
:104280009385070013050700EFC00FE46F000005DA
:1042900097C701009387C72D03A7070097C70100A1
:1042A0009387471483A707009387470093850700E8
:1042B00013050700EFC04FE197C701009387C7318F
:1042C00083A707000327C100637AF70097C701009F
:1042D000938787300327C10023A0E7001300000065
:1042E0008320C1011301010267800000130101FD59
:1042F00023261102930705002324B1002317F100A0
:1043000083278100639E07008357E100939727006E
:1043100013850700EF20C02E930705006F00800073
:1043200083278100232CF10083278101638A070200
:1043300013050006EF20C02C232EA1008327C10106
:10434000638A07008327C1010327810123A8E702AD
:104350006F00400103258101EF20404A6F0080007B
:10436000232E01008327C101638207028327C10135
:1043700003A707038357E1009397270013860700DD
:104380009305500A13050700EF20006A8327C10137
:10439000138507008320C102130101036780000019
:1043A000130101FC232E1102232C81022326A100DC
:1043B0002324B1002322C100232601028327810088
:1043C00083A707006388071C832781002324F10249
:1043D0008327810283A7470003A747008327810221
:1043E00023A2E7008327810203A7470083278102D6
:1043F00093878700631CF7008327810283A7470008
:1044000003A747008327810223A2E70083278102B5
:1044100083A7470083A7C7002322F10283278100D7
:104420002320F1028327010283A7470003A7470047
:104430008327010223A2E7008327010203A7470085
:104440008327010293878700631CF70083270102FB
:1044500083A7470003A747008327010223A2E700A1
:104460008327010283A7470083A7C700232EF100FB
:104470008327C102939757000327C100B307F700B2
:104480000327C10123A0E7008327C10293975700A8
:104490000327C100B307F7000327C1011307470330
:1044A00023A2E7008327C102939757000327C10087
:1044B000B307F7000327C1010327870423A4E700FC
:1044C0008327C102939757000327C100B307F70062
:1044D0000327410023A6E7008327C10293975700D3
:1044E0000327C100B307F7000327C1010327C70251
:1044F00023A8E70003274100930730006314F70265
:104500008327C10183A78702638E07008327C10227
:10451000939757000327C100B307F7001307200044
:1045200023A6E7008327C102939757000327C10002
:10453000B307F7000327C1010327070523AAE700F4
:104540008327C102939757000327C100B307F700E1
:1045500023AC07008327C10183A607038327C10279
:10456000939757000327C1003304F7001385060013
:10457000EF00C00393070500231EF4008327C10248
:10458000938717002326F1020327C10183274102E5
:10459000E316F7E88327C102138507008320C103D0
:1045A000032481031301010467800000130101FE4D
:1045B0002326A100232E01006F00C0018327C10024
:1045C000938717002326F1008327C10193871700E3
:1045D000232EF1008327C10003C707009307500A69
:1045E000E30EF7FC8327C10193D72700232EF100A8
:1045F0008327C1019397070193D70701138507000C
:104600001301010267800000130101FE232E110037
:104610002326A1008327C10083A707031385070072
:10462000EF20C01D0325C100EF20401D1300000036
:104630008320C1011301010267800000130101FF03
:1046400097C701009387C7F283A7070083A70700D6
:1046500063960700930710006F0080009307000027
:10466000638C070097C70100938707F71307F0FFD4
:1046700023A0E7006F00000397C70100938747EF6F
:1046800083A7070083A7C70083A7C7002326F100DD
:104690008327C10003A7470097C701009387C7F38B
:1046A00023A0E70013000000130101016780000050
:1046B000130101FF97C701009387C7D283A70700A3
:1046C0002326F1008327C100138507001301010190
:1046D00067800000130101FF97C70100938787EEF1
:1046E00083A7070063980700930710002326F100B3
:1046F0006F00400297C70100938747EE83A707002A
:1047000063980700930720002326F1006F008000C4
:10471000232601008327C10013850700130101012F
:1047200067800000130101FD232611022326A1004A
:104730008327C100232EF1008327C100638A07125B
:104740008327C10103A7C70297C70100938787C9C1
:1047500083A7070083A7C702637CF7108327C101E3
:1047600083A7870163C2070297C70100938787C7A2
:1047700083A7070083A7C7021307A0003307F740EA
:104780008327C10123ACE7008327C10183A647012A
:104790008327C10103A7C702930707009397270048
:1047A000B387E7009397270017C70100130747CD8A
:1047B000B387E7006396F600930710006F00800050
:1047C00093070000638A07088327C1019387470086
:1047D00013850700EFC0CF9B97C70100938787C061
:1047E00083A7070003A7C7028327C10123A6E70207
:1047F0008327C10103A7C70297C70100938747DC3E
:1048000083A7070063FCE7008327C10103A7C70252
:1048100097C701009387C7DA23A0E7008327C10168
:1048200003A7C7029307070093972700B387E70002
:104830009397270017C70100130787C43387E70042
:104840008327C1019387470093850700130507005D
:10485000EFB0DFFF6F00C00197C70100938787B8F3
:1048600083A7070003A7C7028327C10123A6E70286
:10487000130000008320C1021301010367800000C0
:10488000130101FD232611022326A1008327C10065
:10489000232CF100232E01008327C100638607101B
:1048A00097C70100938707B483A7070003278101F7
:1048B0006306F700737004306F00000083278101E6
:1048C00083A7470563960700737004306F000000EC
:1048D0008327810183A747051387F7FF832781017A
:1048E00023AAE7048327810103A7C7028327810145
:1048F00083A70705630AF70A8327810183A7470572
:104900006394070A83278101938747001385070073
:10491000EFC00F888327810103A707058327810143
:1049200023A6E7028327810183A7C7021307A000FC
:104930003307F7408327810123ACE70083278101F8
:1049400003A7C70297C70100938787C783A70700FC
:1049500063FCE7008327810103A7C70297C7010013
:10496000938707C623A0E7008327810103A7C70217
:104970009307070093972700B387E70093972700D3
:1049800017C701001307C7AF3387E70083278101EB
:10499000938747009385070013050700EFB01FEBCF
:1049A00093071000232EF1008327C1011385070010
:1049B0008320C1021301010367800000737004307B
:1049C00097C70100938707C083A707006384070286
:1049D00097C70100938707A183A7070003A7470490
:1049E0001307170023A2E70497C701009387879F47
:1049F00083A70700130000006780000097C701002D
:104A0000938747BC83A707006384070497C7010007
:104A10009387479D83A7070083A74704638A0702FC
:104A200097C701009387079C83A7070003A7470444
:104A30001307F7FF23A2E70497C701009387879A1C
:104A400083A7070083A747046394070073600430BB
:104A50001300000067800000130101FF97C70100E9
:104A60009387479883A7070083A787012326F10030
:104A700097C701009387079783A7070003A7C7027B
:104A800097C701009387079683A707009306A000A6
:104A90003387E64023ACE7008327C1001385070076
:104AA000130101016780000097C701009387879376
:104AB00083A70700638E070097C70100938787923B
:104AC00083A7070003A747051307170023AAE704D6
:104AD00097C701009387079183A7070013850700F5
:104AE00067800000130101FD232611022326A10087
:104AF0002324B100EFF09FEC97C701009387878EC6
:104B000083A7070083A787056396070897C7010057
:104B10009387478D83A707001307100023AEE70490
:104B2000832781006388070697C701009387878BD7
:104B300083A707009387470013850700EFB05FE561
:104B4000032781009307F0FF6314F70297C7010062
:104B50009387478983A707009387470093850700BA
:104B600017C50100130505A4EFB05FCE6F0040022A
:104B700097C70100938787A483A7070003278100B5
:104B8000B307F700232EF1000325C101EFF04FEA30
:104B9000EFB01FA0EFF09FE6EFF05FE297C70100D4
:104BA0009387478483A7070083A78705232CF100F9
:104BB00083278101638C07028327C100638C070070
:104BC00097C701009387078283A7070023AC0704D8
:104BD0006F00C00197C701009387C78083A70700B4
:104BE00003A787051307F7FF23ACE70497B7010076
:104BF0009387477F83A7070023AE0704EFF01FE0EA
:104C000083278101138507008320C102130101035B
:104C100067800000130101FD232611022326A10055
:104C20002324B1002322C1002320D100EFF01FD99B
:104C300097B701009387077B83A7070003A7C705E2
:104C4000930720006306F70A97B7010093878779D7
:104C500083A7070083A687050327C1001347F7FF33
:104C600033F7E60023ACE70497B701009387877713
:104C700083A707001307100023AEE7048327010072
:104C80006388070697B701009387C77583A7070056
:104C90009387470013850700EFB09FCF03270100DC
:104CA0009307F0FF6314F70297B7010093878773A8
:104CB00083A70700938747009385070017C5010066
:104CC0001305458EEFB09FB86F00400297C70100F3
:104CD0009387C78E83A7070003270100B307F70058
:104CE000232CF10003258101EFF08FD4EFB05F8A10
:104CF000EFF0DFD0EFF09FCC83274100638E0700F9
:104D000097B701009387076E83A7070003A787055E
:104D10008327410023A0E70097B701009387876CA2
:104D200083A7070003A7C705930710006316F700C2
:104D3000232E01006F00C00297B701009387876A96
:104D400083A7070083A68705032781001347F7FF82
:104D500033F7E60023ACE70493071000232EF1009D
:104D600097B701009387076883A7070023AE07045E
:104D7000EFF0DFC88327C101138507008320C1023C
:104D80001301010367800000130101FD23261102B6
:104D90002326A1002324B1002322C1002320D10017
:104DA00093071000232EF1008327C10063960700AC
:104DB000737004306F0000008327C100232CF100C2
:104DC000EFF0DFBF83270100638A0700832781019B
:104DD00003A787058327010023A0E700832781011C
:104DE00083A7C705232AF100832781011307200029
:104DF00023AEE704032741009307400063ECE70874
:104E0000832741001397270097B701009387072056
:104E1000B307F70003A7070097B701009387071FA1
:104E2000B307F700678007008327810103A7870581
:104E3000832781003367F7008327810123ACE704D0
:104E40006F0040058327810183A78705138717001B
:104E50008327810123ACE7046F00C003832781010E
:104E60000327810023ACE7046F00C0020327410140
:104E700093072000630AF70083278101032781003D
:104E800023ACE7046F000001232E01006F008000B7
:104E90001300000003274101930710006316F70A6F
:104EA000832781019387470013850700EFB05FAE2A
:104EB0008327810103A7C70297B701009387477033
:104EC00083A7070063FCE7008327810103A7C702CC
:104ED00097B701009387C76E23A0E700832781015E
:104EE00003A7C7029307070093972700B387E7003C
:104EF0009397270017B70100130787583387E700F8
:104F000083278101938747009385070013050700D6
:104F1000EFB0DF938327810183A7870263860700B1
:104F2000737004306F0000008327810103A7C7025C
:104F300097B701009387074B83A7070083A7C70292
:104F400063F4E700EFB0CFE4EFF05FAB8327C1017C
:104F5000138507008320C10213010103678000004D
:104F6000130101FC232E1102232EA100232CB100DA
:104F7000232AC1002328D1002326E1009307100033
:104F80002326F1028327C101639607007370043062
:104F90006F0000008327C1012324F102EFB08FF6D8
:104FA000930705002322F10283270101638A07008A
:104FB0008327810203A787058327010123A0E70038
:104FC0008327810283A7C7052320F102832781025B
:104FD0001307200023AEE704032741019307400095
:104FE00063ECE708832741011397270097B7010077
:104FF00093870703B307F70003A7070097B70100DC
:1050000093870702B307F7006780070083278102B1
:1050100003A78705832781013367F7008327810270
:1050200023ACE7046F0040058327810283A787052F
:10503000138717008327810223ACE7046F00C003A6
:10504000832781020327810123ACE7046F00C0029C
:105050000327010293072000630AF70083278102D8
:105060000327810123ACE7046F000001232601021E
:105070006F00800013000000032701029307100057
:105080006314F70E8327810283A7870263860700D4
:10509000737004306F00000097B7010093870754C6
:1050A00083A70700639E0706832781029387470033
:1050B00013850700EFB0DF8D8327810203A7C702A6
:1050C00097B701009387C74F83A7070063FCE700EA
:1050D0008327810203A7C70297B701009387474E32
:1050E00023A0E7008327810203A7C70293070700D5
:1050F00093972700B387E7009397270017B701001E
:10510000130707383387E700832781029387470017
:105110009385070013050700EFB04FF36F00C00140
:1051200083278102938787019385070017B50100C4
:1051300013058544EFB08FF18327810203A7C702CF
:1051400097B701009387072A83A7070083A7C702A1
:1051500063FCE7008327C100638807008327C10041
:105160001307100023A0E7008327410213850700DF
:10517000EFB08FD78327C102138507008320C103B7
:105180001301010467800000130101FD23261102B1
:105190002326A1002324B1008327C10063960700C2
:1051A000737004306F0000008327C100232EF100CC
:1051B000EFB04FD593070500232CF1008327C101E1
:1051C00083A7C705232AF1008327C1011307200005
:1051D00023AEE7048327C10183A787051387170040
:1051E0008327C10123ACE704032741019307100083
:1051F0006314F70E8327C10183A787026386070024
:10520000737004306F00000097B701009387073D6B
:1052100083A70700639E07068327C1019387470082
:1052200013850700EFB0CFF68327C10103A7C7029C
:1052300097B701009387C73883A7070063FCE7008F
:105240008327C10103A7C70297B701009387473798
:1052500023A0E7008327C10103A7C7029307070024
:1052600093972700B387E7009397270017B70100AC
:10527000130707213387E7008327C101938747007E
:105280009385070013050700EFB04FDC6F00C001E6
:105290008327C101938787019385070017B5010014
:1052A0001305852DEFB08FDA8327C10103A7C7024D
:1052B00097B701009387071383A7070083A7C70247
:1052C00063FCE70083278100638807008327810050
:1052D0001307100023A0E70083278101138507002F
:1052E000EFB08FC0130000008320C102130101033F
:1052F00067800000130101FD232611022326A1006F
:105300008327C100232CF10083278101639A0700C2
:1053100097B701009387070D83A707006F008000F0
:1053200083278101232CF100EFF04FE983278101CE
:1053300003A7C70593072000631CF700832781019B
:1053400023AE070493071000232EF1006F008000A6
:10535000232E0100EFF08FEA8327C1011385070098
:105360008320C1021301010367800000130101FEC5
:10537000232E110023260100EF00500B97B70100E8
:105380009387072983A70700638A07029308000011
:105390001308000093070000130720009306000085
:1053A0001306004097B501009385C5C81705000096
:1053B0001305852EEFC01FEF2326A1008327C10010
:1053C00063960700737004306F0000008327C100EC
:1053D000138507008320C1011301010267800000CB
:1053E000130101FC232E1102232EA100232CB10056
:1053F000232AC1002328D1002326E100832781012D
:1054000063960700232601026F0080061305C00281
:10541000EF10001F2326A1028327C102638A07041D
:10542000EF00D0008327C1020327C10123A0E700BA
:105430008327C1020327810123ACE7008327C10230
:105440000327410123AEE7008327C102032701019F
:1054500023A0E7028327C1020327C10023A2E7029A
:105460008327C1029387470013850700EFB04FBC25
:105470008327810163960700737004306F0000007A
:105480008327C102138507008320C1031301010490
:1054900067800000130101FC232E1102232EA100BE
:1054A000232CB100232AC1002328D1002326E100A8
:1054B000232601028327C10163960700737004301D
:1054C0006F00000097B701009387871483A7070038
:1054D000638C070A832781012320F102832741017E
:1054E0002322F1028327C1012324F1020327810132
:1054F0009307500063C6E706EFF0CF9D1307050042
:10550000930720006318F70297B7010093874710AD
:1055100083A7070013070102930600000326C100BA
:105520009305070013850700EFB0DF9B2326A10238
:105530006F00800597B701009387870D83A7070049
:1055400013070102930600001306000093050700ED
:1055500013850700EFB01F992326A1026F00C00238
:1055600097B701009387C70A83A7070013070102B3
:105570009306000003260101930507001385070029
:10558000EFB09FF02326A1028327C10213850700F5
:105590008320C1031301010467800000130101FE91
:1055A0002326A1008327C100232EF1008327C100F9
:1055B00063960700737004306F0000008327C101F9
:1055C00083A707001385070013010102678000000D
:1055D000130101FD232611022326A1002324B1007B
:1055E00097B701009387470283A7070083A7C700E7
:1055F00083A7C700232EF1008327C10193874700AB
:1056000013850700EFB0CFB88327C10103A7C701F7
:10561000930710006310F7068327C10103A78701D2
:105620008327C100B307F7008326C100032681004A
:10563000938507000325C101EF00802213070500B1
:10564000930710006318F702130700009306000089
:105650000326C100930500000325C101EFF09FE37D
:10566000232CA10083278101639607007370043007
:105670006F0000008327C10183A747020325C101F2
:10568000E7800700130000008320C102130101031B
:1056900067800000130101FD232611022326A100CB
:1056A0009307810113850700EF00800E232EA100D0
:1056B00083278101938507000325C101EF00C00006
:1056C000EF0000286FF0DFFD130101FD232611021A
:1056D0002326A1002324B100EFD01F989307810156
:1056E00013850700EF004011232EA10083278101BD
:1056F0006396070883278100639207020327C1008E
:105700008327C10163ECE700EFD05F978325C101D8
:105710000325C100EFF0DFEB6F00800683278100D7
:105720006380070297B70100938747EE83A70700BE
:1057300083A7070093B7170093F7F70F2324F1000F
:1057400097B701009387C7EC83A607000327C10022
:105750008327C101B307F740032681009385070023
:1057600013850600EFC01FABEFD05F9193070500D4
:1057700063980700EFA0DFE16F008000EFD01F907B
:10578000130000008320C1021301010367800000A1
:10579000130101FE2326A10097B701009387C7E6F6
:1057A00083A7070083A7070093B7170093F7F70FA6
:1057B000138707008327C10023A0E7008327C100C8
:1057C00083A707006390070297B701009387C7E399
:1057D00083A7070083A7C70083A70700232EF10034
:1057E0006F008000232E01008327C101138507006D
:1057F0001301010267800000130101FD232611023D
:105800002326A100EFD09FA4232EA10097B701006B
:10581000938747E083A707000327C101637CF70054
:10582000EF00C02B8327C1001307100023A0E7005F
:105830006F00C0008327C10023A0070097B70100B5
:10584000938747DD0327C10123A0E7008327C10118
:10585000138507008320C102130101036780000044
:10586000130101FD232611022326A1002324B100E8
:105870002322C1002320D100232E01008327C10051
:105880000327810023A2E7008327C1000327C1006B
:1058900023A8E700032781008327410063E6E7048C
:1058A00003274100832701003307F7408327C10006
:1058B00083A787016368F70093071000232EF10088
:1058C0006F00C00697B70100938747D403A707006E
:1058D0008327C100938747009385070013050700BE
:1058E000EFA09FFE6F008004032741008327010083
:1058F000637EF70003278100832701006368F700B8
:1059000093071000232EF1006F00400297B70100AB
:10591000938787CF03A707008327C100938747009A
:105920009385070013050700EFA01FFA8327C10125
:10593000138507008320C102130101036780000063
:10594000130101FD232611026F00801583278100BA
:1059500063C6071483270101232EF1008327C101A9
:1059600083A74701638A07008327C1019387470004
:1059700013850700EFB0CF8193074100138507001F
:10598000EFF09FE7232CA1008327810013079000ED
:105990006368F7101397270097A701009387076A9A
:1059A000B307F70003A7070097A7010093870769CC
:1059B000B307F700678007000327C1008327C101F1
:1059C00083A78701B307F7000327C10093060700E9
:1059D00003268101938507000325C101EFF05FE8ED
:1059E0001307050093071000631CF70A8327C10102
:1059F00083A747020325C101E78007008327C10170
:105A000003A7C70193071000631CF7080327C10011
:105A10008327C10183A78701B307F700130700009D
:105A20009306000013860700930500000325C101BB
:105A3000EFF05FA6232AA1008327410163920706A6
:105A4000737004306F0000000327C1008327C10179
:105A500023ACE7008327C10183A787016396070072
:105A6000737004306F0000008327C10103A7870112
:105A700083278101B307F700832681010326810173
:105A8000938507000325C101EFF09FDD6F00400102
:105A90000325C101EF0090566F0080001300000045
:105AA00097B701009387C7B683A707001307810044
:105AB00093060000130600009305070013850700F6
:105AC000EFB05FC593070500E39207E813000000FD
:105AD0008320C1021301010367800000130101FD4F
:105AE000232611026F00C00E97B701009387C7B13C
:105AF00083A7070083A7C70083A70700232CF10013
:105B000097B70100938747B083A7070083A7C70013
:105B100083A7C700232AF100832741019387470009
:105B200013850700EFA0DFE68327410183A7470223
:105B300003254101E78007008327410103A7C7012F
:105B4000930710006316F7088327410183A7870195
:105B500003278101B307F7002328F1000327010180
:105B60008327810163F0E7048327410103270101B3
:105B700023A2E700832741010327410123A8E7006F
:105B800097B70100938747A803A707008327410120
:105B9000938747009385070013050700EFA0DFD226
:105BA0006F00000313070000930600000326810125
:105BB0009305000003254101EFF0DF8D2326A100AE
:105BC0008327C10063960700737004306F000000E4
:105BD00097B70100938747A383A7070083A7070010
:105BE000E39407F097B70100938707A283A7070004
:105BF000232EF10097B70100938747A103A7070061
:105C000097B70100938747A023A0E70097B701004B
:105C10009387C79F0327C10123A0E700130000005B
:105C20008320C1021301010367800000130101FFFB
:105C300023261100EFE09FD897B701009387479D77
:105C400083A707006394070A17B501001305459958
:105C5000EFA09FB817B501001305C599EFA0DFB7F6
:105C600097B701009387479A17B701001307479723
:105C700023A0E70097B701009387479917B7010062
:105C80001307479723A0E700130600009305C00001
:105C900013054000EFA09FEC1307050097B7010024
:105CA0009387079723A0E70097B70100938747964C
:105CB00083A7070063960700737004306F0000002D
:105CC00097B701009387C79483A7070063800702F3
:105CD00097B701009387C79383A7070097A5010093
:105CE0009385453813850700EFC0CFC2EFE01FD181
:105CF000130000008320C100130101016780000030
:105D0000130101FD232611022326A1008327C100D0
:105D1000232EF1008327C1006396070073700430BF
:105D20006F000000EFE09FC98327C10183A74701EF
:105D3000B337F00093F7F70F232CF100EFE01FCCFF
:105D400083278101138507008320C102130101030A
:105D500067800000130101FD232611022326A10004
:105D60008327C100232EF1008327C100639607001B
:105D7000737004306F000000EFE05FC48327C1013F
:105D800083A70702232CF100EFE05FC7832781017F
:105D9000138507008320C1021301010367800000FF
:105DA000130101FD232611022326A1002324B100A3
:105DB0008327C100232EF1008327C10063960700CB
:105DC000737004306F000000EFE05FBF8327C101F4
:105DD0000327810023A0E702EFE05FC21300000069
:105DE0008320C1021301010367800000130101FE3B
:105DF000232E11001305C001EF0090002326A100FF
:105E00008327C100638E07008327C10023A00700FA
:105E10008327C1009387470013850700EFA0DF9B0E
:105E20008327C100138507008320C10113010102EC
:105E300067800000130101FC232E11022326A1001C
:105E40002324B1002322C1002320D1008327C100D5
:105E50002324F1022322010203274100B70700FF98
:105E6000B377F70063860700737004306F0000009B
:105E70008327410063960700737004306F000000B1
:105E8000EFE05F8593070500639607008327010015
:105E900063960700930710006F00800093070000CF
:105EA00063960700737004306F000000EFD0CF9A44
:105EB0008327810283A707002320F1028325810025
:105EC0000325C100EF0080410327010283278100E1
:105ED0003367F70083274100B377F70003274100BA
:105EE000631CF7020327010283278100B367F700D1
:105EF0002326F1028327810203A70700832741009D
:105F000093C7F7FF3377F7008327810223A0E700C9
:105F1000232001006F0040048327010063880702EB
:105F2000832781029386470003274100B7070005B6
:105F3000B367F70003260100938507001385060069
:105F4000EFD0DFA4232601026F0000018327810226
:105F500083A707002326F102EFD04F92232EA10042
:105F600083270100638407088327C1016394070026
:105F7000EFA00FE2EFE05FAE2326A1020327C102EC
:105F8000B7070002B377F70063980704EFE01FA399
:105F90008327810283A707002326F1020327C1027A
:105FA00083274100B377F700032741006310F7020E
:105FB0008327810203A707008327410093C7F7FFC8
:105FC0003377F7008327810223A0E700EFE01FA3C8
:105FD000930710002322F1020327C102B707000133
:105FE0009387F7FFB377F7002326F1028327C102D7
:105FF000138507008320C10313010104678000009B
:10600000130101FB23261104232EA100232CB10030
:10601000232AC1002328D1002326E1008327C101C0
:10602000232AF102232C0102232801028327C10124
:1060300063960700737004306F000000032781012E
:10604000B70700FFB377F70063860700737004306B
:106050006F0000008327810163960700737004308E
:106060006F000000EFE00FE793070500639607005D
:106070008327C10063960700930710006F0080001C
:106080009307000063960700737004306F000000F0
:10609000EFC09FFC8327410383A707002326F1025B
:1060A00003260101832581010325C102EF00404B36
:1060B0002324A10283278102638C07028327C10264
:1060C000232EF1022326010083274101638807085C
:1060D0008327410303A707008327810193C7F7FFA5
:1060E0003377F7008327410323A0E7006F00000701
:1060F0008327C100639807008327C102232EF10282
:106100006F00C00583274101638A070003278103CD
:10611000B7070001B367F700232CF10283270101C1
:10612000638A070003278103B7070004B367F700FA
:10613000232CF10283274103938647000327810123
:1061400083278103B367F7000326C1009385070007
:1061500013850600EFD09F83232E0102EFC01FF2AC
:106160002322A1028327C1006388070883274102F5
:1061700063940700EFA0CFC1EFE01F8E232EA10292
:106180000327C103B7070002B377F700639C070436
:10619000EFE0DF828327410383A70700232EF1026C
:1061A00003260101832581010325C103EF00403B44
:1061B0009307050063840702832741016380070278
:1061C0008327410303A707008327810193C7F7FFB4
:1061D0003377F7008327410323A0E700EFE01F8216
:1061E000232801020327C103B70700019387F7FFA4
:1061F000B377F700232EF1028327C103138507002D
:106200008320C1041301010567800000130101FD13
:10621000232611022326A1002324B1008327C100D5
:10622000232EF1008327C1006396070073700430AA
:106230006F00000003278100B70700FFB377F70066
:1062400063860700737004306F000000EFE00FF703
:106250008327C10183A70700232CF1008327C101F5
:1062600003A707008327810093C7F7FF3377F70061
:106270008327C10123A0E700EFE04FF883278101C6
:10628000138507008320C10213010103678000000A
:10629000130101FD232611022326A1008327C1003B
:1062A000232EF100EFA00FC693070500232CF10069
:1062B0008327C10183A70700232AF10083278101D7
:1062C00013850700EFA04FC2832741011385070004
:1062D0008320C1021301010367800000130101FB49
:1062E000232611042326A1002324B100232C01021C
:1062F0008327C1002328F102232A01028327C1003A
:1063000063960700737004306F000000032781005C
:10631000B70700FFB377F700638607007370043098
:106320006F00000083270103938747002326F102B3
:106330008327C102938787002324F102EFC0DFD1B6
:106340008327C10283A7C700232EF10283270103FD
:1063500003A70700832781003367F7008327010322
:1063600023A0E7006F00000E8327C10383A7470027
:106370002322F1028327C10383A707002320F10210
:10638000232A010203270102B70700FFB377F700B2
:10639000232EF10003270102B70700019387F7FFBF
:1063A000B377F7002320F1020327C101B7070004E8
:1063B000B377F700639207028327010303A707005F
:1063C00083270102B377F700638807029307100061
:1063D000232AF1026F0040028327010303A707006D
:1063E00083270102B377F700032701026316F70042
:1063F00093071000232AF1028327410363800704D7
:106400000327C101B7070001B377F700638A0700CC
:106410000327810383270102B367F700232CF102CE
:106420008327010303A70700B7070002B367F7003C
:10643000938507000325C103EFD05F8283274102C4
:10644000232EF1020327C10383278102E31EF7F005
:106450008327010303A707008327810393C7F7FF5F
:106460003377F7008327010323A0E700EFC01FC1A4
:106470008327010383A70700138507008320C10436
:106480001301010567800000130101FD232611029D
:106490002326A1008327C100232EF1008327C101F9
:1064A00093874700232CF100EFC01FBB6F00400310
:1064B0008327810103A7C700832781019387870072
:1064C0006316F700737004306F00000083278101AA
:1064D00083A7C700B705000213850700EFD00FF8A8
:1064E0008327810183A70700E39407FC0325C101EB
:1064F000EF00C030EFC09FB8130000008320C1023E
:106500001301010367800000130101FE232E110017
:106510002326A1002324B100832581000325C10087
:10652000EFF0DFDB130000008320C1011301010243
:1065300067800000130101FE232E11002326A10015
:106540002324B100832581000325C100EFF01FCC77
:10655000130000008320C1011301010267800000C5
:10656000130101FE2326A1002324B1002322C10030
:10657000232E010083274100639007020327C100F7
:1065800083278100B377F700638607029307100023
:10659000232EF1006F0000020327C1008327810032
:1065A000B377F700032781006316F7009307100005
:1065B000232EF1008327C101138507001301010277
:1065C00067800000130101FE2326A1008327C1007C
:1065D000232CF1008327C10063960700232E0100BE
:1065E0006F0000018327810183A78701232EF1001B
:1065F0008327C10113850700130101026780000092
:10660000130101FC232E11022326A10023220102E3
:10661000EFC09FA4973703009387070183A7070064
:10662000639C0700EF00002C973703009387C7FF98
:106630001307100023A0E7008327C100638A070225
:1066400093078000138707008327C100B387E70003
:106650002326F1008327C10093F73700638A0700E0
:106660008327C10093F7C7FF938747002326F100D4
:106670008327C100638207160327C100B797010073
:106680009387B7FF63EAE714973703009387C7F848
:106690002324F10297370300938707F883A70700A5
:1066A0002326F1026F0080018327C1022324F10217
:1066B0008327C10283A707002326F1028327C10293
:1066C00083A747000327C10063F8E7008327C102BF
:1066D00083A70700E39A07FC0327C102973703004B
:1066E000938707F4630AF70E8327810283A70700C5
:1066F00013078000B387E7002322F1028327C1023A
:1067000003A707008327810223A0E7008327C10294
:1067100003A747008327C100B307F7401307800092
:10672000131717006378F7080327C1028327C100F6
:10673000B307F700232EF1008327C10203A7470008
:106740008327C1003307F7408327C10123A2E70055
:106750008327C1020327C10023A2E7008327C101C9
:1067600083A74700232CF100973703009387C7EADC
:106770002320F1026F0000018327010283A7070095
:106780002320F1028327010283A7070083A7470084
:1067900003278101E3E2E7FE8327010203A7070045
:1067A0008327C10123A0E700832701020327C1013A
:1067B00023A0E70097A70100938707C403A707005A
:1067C0008327C10283A747003307F74097A701003B
:1067D000938787C223A0E700EFC05F8A8327410227
:1067E00063940700EF10C017832741021385070049
:1067F0008320C1031301010467800000130101FD20
:10680000232611022326A1008327C100232CF10097
:106810008327C1006382070A93078000B307F04013
:1068200003278101B307F700232CF100832781019F
:10683000232AF100EFC05F828327410183A747002D
:106840002328F10097370300938707DD232EF100FB
:106850006F0000018327C10183A70700232EF100E9
:106860008327C10183A7070083A7470003270101EE
:10687000E3E2E7FE8327C10103A707008327410165
:1068800023A0E7008327C1010327410123A0E700DC
:106890008327410103A7470097A701009387C7B546
:1068A00083A707003307F70097A701009387C7B4B2
:1068B00023A0E700EFC08FFC130000008320C1027B
:1068C000130101036780000097A701009387C7B2F7
:1068D00083A70700138507006780000013000000EE
:1068E00067800000130101FF97A70100938707D37A
:1068F00093F7C7FF2326F100973703009387C7D18B
:106900000327C10023A0E700973703009387C7D070
:1069100023A2070097370300938787D0379701009A
:106920001307C7FF23A2E70097370300938747CFDA
:1069300023A007008327C1002324F10083278100BF
:10694000379701001307C7FF23A2E70083278100C1
:10695000173703001307C7CC23A0E700130000007C
:106960001301010167800000130101FE2326A1002D
:106970002324B1002322C10083278100232EF100AC
:106980008327C100232CF1000327C1008327810046
:10699000B367F70093F73700639607066F00C002EE
:1069A0008327C10103A707008327810123A0E700F4
:1069B0008327810193874700232CF1008327C1019E
:1069C00093874700232EF100832741009387D7FF49
:1069D0000327C100B307F70003278101E362F7FC37
:1069E0006F0040020327C10193071700232EF10017
:1069F0008327810193861700232CD10003470700CA
:106A00002380E7000327C10083274100B307F70075
:106A100003278101E368F7FC8327C1001385070082
:106A20001301010267800000130101FE2326A1006B
:106A30002324B1002322C1000327C1008327410082
:106A4000B367F70093F73700639807068327810041
:106A500093F7F70F232AF1008327410193978700CB
:106A600003274101B367F700232AF100832741017F
:106A70009397070103274101B367F700232AF10029
:106A80008327C100232EF1006F0080018327C101FD
:106A900013874700232EE1000327410123A0E700CD
:106AA0000327C10083274100B307F7000327C10173
:106AB000E36EF7FC6F00C0038327C100232CF100B5
:106AC0006F00C0018327810113871700232CE10089
:106AD000032781001377F70F2380E7000327C10006
:106AE00083274100B307F70003278101E36CF7FC1C
:106AF0008327C1001385070013010102678000008E
:106B0000130101FE2326A1008327C100232EF100DB
:106B10006F0000018327C10193871700232EF10026
:106B20008327C10183C70700E39607FE0327C1013E
:106B30008327C100B307F740138507001301010243
:106B400067800000130101FE2326A1002324B10069
:106B50008327C100138717002326E10083C707009E
:106B6000A30FF10083278100138717002324E1007E
:106B700083C70700230FF1008347F10163880700F3
:106B80000347F1018347E101E304F7FC0347F10107
:106B90008347E101B307F7401385070013010102A2
:106BA00067800000130101FE2326A1002324B10009
:106BB0008327C100232EF10013000000032781006A
:106BC000930717002324F1008327C1019386170040
:106BD000232ED100034707002380E70083C7070067
:106BE000E39E07FC8327C100138507001301010200
:106BF00067800000130101FE2326A100232E01005F
:106C0000232C01006F0000018327C1009387170028
:106C10002326F1008327C10003C707009307000262
:106C2000E304F7FE8327C10003C707009307D002E0
:106C3000630AF7008327C10003C707009307B00268
:106C40006312F7068327C10083C70700938737FDC8
:106C500093B7170093F7F70F232CF1008327C10098
:106C6000938717002326F1006F00C0030327C1019B
:106C70009307070093972700B387E70093971700C0
:106C8000232EF1008327C100138717002326E1007C
:106C900083C70700938707FD0327C101B307F700E8
:106CA000232EF1008327C10083C70700E39007FC70
:106CB00083278101638807008327C101B307F04060
:106CC0006F0080008327C1011385070013010102B3
:106CD00067800000130101FE2326A10097370300FF
:106CE0009387479683A707009386170017370300FB
:106CF000130747952320D7000327C1001377F70F09
:106D00009736030093860698B387F6002380E70042
:106D10000327C1009307A000630CF7009737030017
:106D20009387479203A7070093070004631EF704A5
:106D30009737030093870795232EF1006F00C00358
:106D40008327C10113871700232EE10003C7070023
:106D5000B70710F0938707F023A0E70097370300E9
:106D60009387478E83A707001387F7FF97370300A2
:106D70009387478D23A0E700973703009387878C7D
:106D800083A70700E39E07FA930700001385070017
:106D90001301010267800000130101EB2326111487
:106DA000232481142322911423202115232E31130F
:106DB000232C4113232A5113232EA100232CB1008D
:106DC0002328C100232AD1002326E1002324F10037
:106DD00023220101232601128327C100138A070001
:106DE000930A0000832701010328410113060A00CA
:106DF00093860A001385070093050800EF1090237F
:106E00009307050013880500138607009306080002
:106E10008327C112138717002326E11213070600E8
:106E20009397270093060113B387F60023AEE7EE8E
:106E30008327C100138407009304000083274101C6
:106E40001387040063E8E7048327410113870400E4
:106E50006398E700832701011307040063ECE7024E
:106E60008327C10013890700930900001306090056
:106E7000938609000325010183254101EF10C03DE0
:106E800093070500138805002328F100232A010138
:106E90006FF09FF4130000006F0040018327C101D1
:106EA0008325810103254100E780070083278100B6
:106EB0001387F7FF2324E1000327C112E340F7FE05
:106EC0006F0040058327C112939727001307011312
:106ED000B307F70003A7C7EF8327C11293972700D3
:106EE00093060113B387F60083A6C7EF93079000BC
:106EF00063F6D700930770056F00800093070003C7
:106F0000B387E7000327C1018325810113850700AB
:106F1000E70007008327C1121387F7FF2326E1123A
:106F2000E342F0FA130000008320C114032481140B
:106F300083244114032901148329C113032A8113D3
:106F4000832A41131301011567800000130101FF1B
:106F50002326A1002324B1008326810013071000FB
:106F60006356D7028327C10083A707009387770062
:106F700093F787FF938687000327C1002320D7005C
:106F800003A8470083A707006F00000503278100BF
:106F9000630407020327C100032707001306470005
:106FA0008326C10023A0C60003270700930707001C
:106FB000130800006F0040020327C10003270700E9
:106FC000130647008326C10023A0C600032707003D
:106FD00093070700130800001385070093050800B6
:106FE0001301010167800000130101FF2326A100A6
:106FF0002324B10083268100130710006356D702B3
:107000008327C10083A707009387770093F787FF43
:10701000938687000327C1002320D70003A84700D9
:1070200083A707006F00800503278100630607021E
:107030000327C10003270700130647008326C1006A
:1070400023A0C60003270700930707001357F74143
:10705000130807006F0080020327C1000327070001
:10706000130647008326C10023A0C600032707009C
:10707000930707001357F74113080700138507000C
:10708000930508001301010167800000130101FC52
:10709000232E1102232C8102232A91022326A100F0
:1070A0002324B1002322C1002320D1006F0040021D
:1070B0006300043C83274100938717002322F100DB
:1070C0008327C1008325810013050400E7800700A2
:1070D0008327410083C707001384070093075002EA
:1070E000E318F4FC83274100938717002322F10063
:1070F000832741002328F10093070002A30BF1002E
:107100009307F0FF232EF1009307F0FF232CF100EB
:107110002320010283274100138717002322E10067
:1071200083C70700138407009307D4FD1307500596
:107130006360F7321397270097970100938787F3CF
:10714000B307F70003A7070097970100938787F21B
:10715000B307F700678007009307D002A30BF10085
:107160006FF05FFB93070003A30BF1006FF09FFA32
:10717000232C010003278101930707009397270021
:10718000B387E70093971700B307F400938707FDD1
:10719000232CF1008327410083C7070013840700D5
:1071A0009307F00263D287049307900363CE8702AC
:1071B00083274100938717002322F1006FF09FFB84
:1071C00083270100138747002320E10083A70700DE
:1071D000232CF1006F0080018327C101E3DC07F25B
:1071E000232E01006FF01FF3130000008327C1015D
:1071F000E3D207F283278101232EF1009307F0FFEA
:10720000232CF1006FF01FF18327010293871700F1
:107210002320F1026FF01FF083270100138747003E
:107220002320E10083A707000327C10083258100F5
:1072300013850700E70007006F0040238327010044
:10724000138747002320E10083A40700639604000E
:1072500097940100938484E18327C1016350F0086F
:10726000034771019307D002630AF7068327810160
:107270009385070013850400EF00D07B13070500FA
:107280008327C101B387E740232EF1006F0040023E
:10729000834771010327C1008325810013850700FF
:1072A000E70007008327C1019387F7FF232EF10032
:1072B0008327C101E34EF0FC6F0040028327C10029
:1072C0008325810013050400E780070093841400E0
:1072D0008327C1019387F7FF232EF10083C70400A2
:1072E000138407006300040483278101E3C807FCBB
:1072F000832781019387F7FF232CF10083278101E6
:10730000E3DE07FA6F0000028327C10083258100B6
:1073100013050002E78007008327C1019387F7FF69
:10732000232EF1008327C101E340F0FE6F0000141B
:10733000930701008325010213850700EFF0DFCAE0
:1073400093070500138805002324F1022326010377
:10735000832781020328C1029307080063D607042C
:107360008327C100832581001305D002E780070031
:10737000832581020326C102930700001308000041
:10738000B386B7401385060033B5A7003307C8405E
:10739000B307A74013870700938706001308070069
:1073A0002324F102232601039307A0002322F102E4
:1073B0006F0040069307A0002322F1026F00000433
:1073C000930780002322F1026F004003930710000F
:1073D0002320F1028327C1008325810013050003C8
:1073E000E78007008327C1008325810013058007FC
:1073F000E7800700930700012322F10293070100B1
:107400008325010213850700EFF05FB42324A10256
:107410002326B10203274102834771011388070025
:107420008327C101032681028326C10283258100AF
:107430000325C100EFF05F966F0040038327C10072
:107440008325810013050400E78007006F00000218
:107450008327C1008325810013055002E7800700C0
:10746000832701012322F100130000006FF05FC6A3
:10747000130000008320C1030324810383244103FC
:107480001301010467800000130101FF2326A100FE
:10749000B70710F0938707F20327C10023A0E70086
:1074A0006F000000130101FB232611022326A10017
:1074B000232AB102232CC102232ED1022320E1046E
:1074C0002322F10423240105232611059307010536
:1074D000938747FE232EF1008327C101938607007F
:1074E0000326C1009305000017F5FFFF1305C57EB5
:1074F000EFF0DFB993070000138507008320C10276
:107500001301010567800000130101FE2326A1007D
:107510002324B1002322710083278100232EF10050
:107520008327C10183A707000327C1001377F70F43
:107530002380E7008327C10183A707001387170073
:107540008327C10123A0E7001300000013010102FB
:1075500067800000130101FA232E11022326A100E7
:107560002324B1002324C1042326D1042328E104C9
:10757000232AF104232C0105232E1105930701066C
:107580002322F102930741019305410117060000F0
:107590001306C6F737F7FFFF9346F7FF37150000CE
:1075A000130505803388A5003378E8001368783B1D
:1075B00023A007013305A6003377E500136777336F
:1075C00023A2E70033F7D50093154701378703005F
:1075D0001307373933E7E50023A4E7003377D600F4
:1075E00093164701370703001307770633E7E600D2
:1075F00023A6E7000F1000008327C1002326F10215
:1076000093070106938787FE2324F1020327810253
:1076100093074101138507009307C10093060700F4
:107620000326810093850700EFF05FA68327C10042
:10763000238007008327C100138707008327C10227
:10764000B307F740138507008320C1031301010628
:1076500067800000130101FF370510F0130545F4A2
:10766000032505002326A100370510F0130505F4B6
:10767000032505002324A100370510F0130545F468
:10768000032505008328C100E398A8FC0325C10059
:107690001303050093030000131703009306000073
:1076A000032581009305050013060000B3E7B6002B
:1076B0003368C700370710F0130587F49305007D82
:1076C00013060000B386B70093880600B3B8F8002D
:1076D0003307C800B387E8001387070093870600C5
:1076E000130807002320F5002322050113000000E2
:1076F0001301010167800000130101FF232611001F
:10770000EFF05FF59307000873A047301300000007
:107710008320C1001301010167800000130101FEF5
:10772000232E11002326A10017950100130505AA99
:10773000EFF05FD7130000008320C10113010102A5
:1077400067800000130101FE232E11002326A100F3
:1077500017950100130505A8EFF0DFD41300000012
:107760008320C1011301010267800000130101FDA4
:10777000232611022326A100232E01006F004001C1
:10778000130000008327C10193871700232EF10007
:107790000327C101B717000093877738E3D2E7FECC
:1077A00017950100130585A3EFF0DFCF6FF0DFFC25
:1077B000130101FF23261100EF00C01C130000007D
:1077C0008320C1001301010167800000130101FE45
:1077D000232E110023260100EF00901B1307050044
:1077E00093071000630EF700179501001305859F9E
:1077F000EFF05FCB8327C10093E727002326F1003A
:107800008327C100138507008320C10113010102F2
:1078100067800000130101FE232E110023260100C2
:10782000EFF01FF917070000130787069306000003
:107830001306100093054006179501001305459C9B
:10784000EFD01FBA2326A1008327C100638207025D
:10785000EFB0DF9F930705001307000093060000B9
:1078600013860700930510000325C100EFD09FC2C7
:1078700023240100EFB08FF0930700001385070069
:107880008320C1011301010267800000130101FD83
:10789000232611022326A100979701009387C7B4DE
:1078A00083A7070013874706979701009387C7B3FD
:1078B00023A0E70097970100938747B383A70700AA
:1078C0001387470697970100938747B223A0E700E5
:1078D00097970100938747B103A70700B7170000E8
:1078E000938777BB63D2E706979701009387C7AF6B
:1078F00003A70700B7F7FFFF938787443307F70015
:1079000097970100938747AE23A0E700EFF01FECA5
:10791000232EA1008327C101639E070097970100D2
:107920009387C7AC03A70700B72700009387773278
:1079300063D0E7028327C10113850700EFF0DFB4AE
:10794000EFB0CFEE6F000001130000006F00800069
:10795000130000008320C1021301010367800000AF
:10796000737004306F000000130000006780000097
:10797000130101FF2326A1002324B10073700430FA
:107980006F000000130101FF232611001306000001
:107990009305400013055000EF904F9C130705001E
:1079A00097270300938707D223A0E70097270300B8
:1079B000938747D183A70700979501009385058595
:1079C00013850700EFA00FF59308000013080000CF
:1079D00093070000130730009306000013060040D1
:1079E0009795010093858583170500001305C5044D
:1079F000EFA05F8B93080000130800009727030097
:107A0000938787CC130720009306000013060040DD
:107A10009795010093850581170500001305855C86
:107A2000EFA05F88130000008320C1001301010153
:107A300067800000130101FC232E11022326A10000
:107A4000232001026F00C00B832701021307A0004F
:107A5000B317F7002326F102EFC05FF6EFB00FFF78
:107A60002324A102972703009387C7C583A7070094
:107A70001307C101930600000326C1029305070006
:107A800013850700EF909F8093070500638A070026
:107A900097270300938707C41307100023A0E7006C
:107AA000EFB0CFFA1307050083278102B307F74031
:107AB0002322F102EFC09FF4032741028327C10272
:107AC000637AF700972703009387C7C01307100056
:107AD00023A0E7008327C1029387C7000327410241
:107AE00063FAE700972703009387C7BE13071000C8
:107AF00023A0E70083270102938717002320F102C8
:107B00000327010293074000E3D0E7F4232001029A
:107B10006F000005972703009387C7BA83A7070064
:107B200013070102930600001306000093050700E7
:107B300013850700EF900FDF130705009307100070
:107B4000630AF700972703009387C7B8130710004D
:107B500023A0E70083270102938717002320F10267
:107B60000327010293074000E3D6E7FA232001022E
:107B70006F00C00B832701021307A000B317F700A3
:107B80002326F102EFC09FE3EFB04FEC2324A102C4
:107B900097270300938707B383A707001307010202
:107BA000930600000326C102930507001385070012
:107BB000EF904FD793070500638A070097270300CC
:107BC000938747B11307100023A0E700EFB00FE839
:107BD0001307050083278102B307F7402322F10230
:107BE000EFC0DFE1032741028327C102637AF70078
:107BF00097270300938707AE1307100023A0E70021
:107C00008327C1029387C7000327410263FAE70075
:107C100097270300938707AC1307100023A0E70002
:107C200083270102938717002320F1020327010213
:107C300093074000E3D0E7F4972703009387C7A991
:107C400023A0070097270300938707A883A70700AF
:107C500013850700EFB0CF8F6F00C0001305400100
:107C6000EFA05FB097270300938707A703A707003C
:107C700093075005E314F7FE13054001EFA09FAEF4
:107C800097270300938747A523A00700232001021D
:107C90006F008010972703009387C7A283A7070070
:107CA0001307C101930600001306000093050700A7
:107CB00013850700EF908FDD130705009307100071
:107CC000630AF700972703009387C7A013071000E4
:107CD00023A0E700972703009387C79E83A7070089
:107CE0001307010293060000130600009305070026
:107CF00013850700EF900FC31307050093071000CB
:107D0000630AF700972703009387C79C13071000A7
:107D100023A0E700972703009387079C03A707008A
:107D200093075005631AF700972703009387879AF4
:107D30001307100023A0E700972703009387C79835
:107D400083A707009305500013850700EFA05FC5C8
:107D5000972703009387479803A7070093075005C9
:107D6000631AF700972703009387C796130710003D
:107D700023A0E700972703009387079583A70700B1
:107D80009305200013850700EFA09FC18327010200
:107D9000938717002320F102032701029307400075
:107DA000E3DAE7EE6F00C00013054001EFA09F9BF0
:107DB000972703009387479203A70700930750056F
:107DC000E314F7FE13054001EFA0DF9997270300A6
:107DD0009387879023A00700232001026F000005EE
:107DE000972703009387078E83A707001307C10116
:107DF0009306000013060000930507001385070093
:107E0000EF90CFC81307050093071000630AF7002F
:107E1000972703009387078C1307100023A0E70020
:107E200083270102938717002320F1020327010211
:107E300093074000E3D6E7FA972703009387C788A4
:107E400083A7070013850700EFA09FF06F00C00015
:107E500013054001EFA01F91972703009387C78761
:107E600003A7070093075005E314F7FE130540012D
:107E7000EFA05F8F972703009387078623A0070053
:107E8000232001026F0080109727030093878783C8
:107E900083A70700130701029306000013060000E2
:107EA0009305070013850700EF90CFA71307050080
:107EB00093071000630AF7009727030093878781D1
:107EC0001307100023A0E700971703009387877F0D
:107ED00083A707001307C1019306000013060000E3
:107EE0009305070013850700EF904FBA13070500AD
:107EF00093071000630AF700971703009387877DA5
:107F00001307100023A0E700971703009387C77C8F
:107F100003A7070093075005631AF700971703009C
:107F20009387477B1307100023A0E70097170300F0
:107F30009387877983A7070093055000138507006F
:107F4000EFA01FA6971703009387077903A70700E1
:107F500093075005631AF7009717030093878777F5
:107F60001307100023A0E700971703009387C77536
:107F700083A707009305200013850700EFA05FA2E9
:107F800083270102938717002320F10203270102B0
:107F900093074000E3DAE7EE6F00C00013054001ED
:107FA000EFA04FFC971703009387077303A7070001
:107FB00093075005E314F7FE13054001EFA08FFA75
:107FC000971703009387877083A70700138717000D
:107FD000971703009387876F23A0E7006FF05FA6D2
:107FE000130101FD232611022326A1001305000021
:107FF000EFA05FBBEFC09F9CEFB04FA5232EA10069
:10800000232A0100971703009387076D1307500574
:1080100023A0E700971703009387C76A83A7070089
:1080200013074101930600001306F00A93050700A9
:1080300013850700EF900F8F93070500638A0700F1
:1080400097170300938707691307100023A0E70021
:10805000EFB0CF9F130705008327C101B307F74097
:10806000232CF100EFC09F99032781019307E00AB9
:1080700063EAE700971703009387C76513071000AB
:1080800023A0E700032781019307B00B63FAE70001
:1080900097170300938707641307100023A0E700D6
:1080A00097170300938747631307500523A0E70042
:1080B00013050000EFA01FAFEFC05F90EFB00F9966
:1080C000232EA1009717030093870761130750051C
:1080D00023A0E700971703009387C75E83A70700D5
:1080E00013074101930600001306F00A93050700E9
:1080F00013850700EF908F9993070500638A0700A7
:10810000971703009387075D1307100023A0E7006C
:10811000EFB0CF93130705008327C101B307F740E2
:10812000232CF100EFC09F8D032781019307E00A04
:1081300063EAE700971703009387C75913071000F6
:1081400023A0E700032781019307B00B63FAE70040
:1081500097170300938707581307100023A0E70021
:1081600097170300938747571307500523A0E7008D
:10817000971703009387C75583A707001387170036
:10818000971703009387C75423A0E7006FF01FE6FB
:10819000130101FF930710002326F1009717030036
:1081A0009387C75203A707009717030093870753C6
:1081B00083A707006314F700232601009717030025
:1081C0009387075103A70700971703009387475129
:1081D00083A707006314F700232601009717030005
:1081E0009387474F03A70700930710006314F70016
:1081F00023260100971703009387874D03A70700E5
:10820000971703009387C74D23A0E7009717030034
:108210009387C74B03A70700971703009387074C63
:1082200023A0E7008327C100138507001301010184
:1082300067800000B305B500930705006386B700AB
:1082400003C70700631607003385A7406780000057
:10825000938717006FF09FFE130101FD2322910207
:10826000232A5101232611022324810223202103E2
:10827000232E3101232C4101232861012326710182
:1082800023248101232291012320A101930A0500C7
:1082900093840500639E06381304060093090500C5
:1082A00017890100130989F863F8C512B70701009F
:1082B000138B05006378F6101307F00F3337C700F0
:1082C00013173700B357E6003309F9008346090056
:1082D0003387E60093060002B386E640638C06000F
:1082E000B394D40033D7EA003314D600336B97002D
:1082F000B399DA00935A040193850A0013050B0021
:10830000EF00902A1309050093850A00931B0401CE
:1083100013050B00EF00D02493DB0B019304050041
:108320009305050013850B00EF00D02013190901F8
:1083300093D70901B367F900138A040063FEA7000D
:10834000B3878700138AF4FF63E8870063F6A7000A
:10835000138AE4FFB3878700B384A74093850A009C
:1083600013850400EF0050241309050093850A00CB
:1083700013850400EF00D01E9399090193040500B2
:10838000930505001319090113850B0093D9090101
:10839000EF00501AB36939011386040063FCA90089
:1083A000B30934011386F4FF63E6890063F4A9007E
:1083B0001386E4FF13140A013364C400130A000097
:1083C0006F000013B707000113070001E36CF6EE1E
:1083D000130780016FF01FEF138A0600631A06006F
:1083E0009305000013051000EF009017130405001B
:1083F000B7070100637EF4129307F00F63F4870060
:10840000130A8000B35744013309F90003470900F8
:108410009306000233074701B386E64063940612D1
:10842000B3848440130A1000135B040193050B000E
:1084300013850400EF0050171309050093050B0086
:1084400013850400931B0401EF00901193DB0B01D3
:10845000930405009305050013850B00EF00900DB4
:108460001319090193D70901B367F900938A04002E
:1084700063FEA700B3878700938AF4FF63E8870051
:1084800063F6A700938AE4FFB3878700B384A7400D
:1084900093050B0013850400EF001011130905006C
:1084A00093050B0013850400EF00900B93990901CD
:1084B00093040500930505001319090113850B00AA
:1084C00093D90901EF001007B3693901138604003D
:1084D00063FCA900B30934011386F4FF63E6890045
:1084E00063F4A9001386E4FF13940A013364C40003
:1084F0001305040093050A008320C10203248102AE
:1085000083244102032901028329C101032A810135
:10851000832A4101032B0101832BC100032C81001D
:10852000832C4100032D010013010103678000002B
:10853000B7070001130A0001E366F4EC130A800197
:108540006FF05FEC3314D40033DAE400B399DA004F
:1085500033D7EA00935A0401B394D40093850A00F8
:1085600013050A00336B9700EF0010041309050090
:1085700093850A0013050A00931B0401EF00407E57
:1085800093DB0B01930405009305050013850B0095
:10859000EF00407A1319090113570B013367E90003
:1085A000138A0400637EA70033078700138AF4FF51
:1085B000636887006376A700138AE4FF33078700A8
:1085C000B304A74093850A0013850400EF00C07D23
:1085D0001309050093850A0013850400EF00407815
:1085E000930405009305050013850B00EF008074CC
:1085F00013170B011357070113190901B367E9009A
:108600001387040063FEA700B38787001387F4FF76
:1086100063E8870063F6A7001387E4FFB38787004A
:10862000131A0A01B384A740336AEA006FF0DFDF50
:1086300063ECD51EB707010063F4F6041307F00FCF
:10864000B335D7009395350033D7B600978701002F
:108650009387C7BDB387E70003C70700130A00026B
:108660003307B700330AEA4063160A021304100006
:10867000E3E096E833B6CA00134416006FF05FE7F4
:10868000B707000193050001E3E0F6FC93058001C4
:108690006FF09FFBB35CE600B3964601B3ECDC00E1
:1086A00033D4E40093DB0C01B397440133D7EA00E1
:1086B00093850B0013050400336BF700B3194601D3
:1086C000EF00806E1309050093850B00130504006D
:1086D000139C0C01EF00C068135C0C0193040500AF
:1086E0009305050013050C00EF00C0641319090180
:1086F00013570B013367E90013840400637EA7005E
:10870000330797011384F4FF636897016376A7002A
:108710001384E4FF33079701B304A74093850B004C
:1087200013850400EF0040681309050093850B00D2
:1087300013850400EF00C062930405009305050053
:1087400013050C00EF00005F93170B0113190901CB
:1087500093D70701B367F9001386040063FEA700EF
:10876000B38797011386F4FF63E8970163F6A700C8
:108770001386E4FFB387970113140401B70B0100BC
:108780003364C4001389FBFF337D240133F92901CD
:10879000B384A7409305090013050D00EF0080592D
:1087A000935C040193050900130B050013850C006D
:1087B000EF00405893D90901130C05009385090077
:1087C00013850C00EF00005713090500938509007D
:1087D00013050D00EF0000563305850193570B017B
:1087E0003385A70063748501330979019357050127
:1087F000B387270163E6F402E392F4BCB7070100F4
:108800009387F7FF3375F50013150501337BFB00E4
:1088100033964A0133056501130A0000E37AA6CCBA
:108820001304F4FF6FF09FB9130A00001304000053
:108830006FF01FCC130101FB232481042322910438
:10884000232E310323229103232611042320210503
:10885000232C4103232A5103232861032326710378
:10886000232481032320A103232EB101930C0500AF
:10887000938905001304050093840500639E062672
:1088800013090600138A0600978A0100938A0A9A40
:1088900063F4C514B70701006376F6129307F00F6F
:1088A00063F4C700130A8000B3574601B38AFA0085
:1088B00003C70A001305000233074701330AE540E6
:1088C000630C0A00B395490133D7EC003319460114
:1088D000B364B70033944C01935A090193850A009D
:1088E00013850400EF00404C9309050093850A00AE
:1088F000131B090113850400EF008046135B0B0175
:108900009305050013050B00EF00C0429399090180
:1089100093570401B3E7F90063FAA700B38727016F
:1089200063E6270163F4A700B3872701B384A74058
:1089300093850A0013850400EF00004793090500A2
:1089400093850A0013850400EF008041131404018D
:10895000930505009399090113050B0013540401B5
:10896000EF00403D33E48900637AA400330424011E
:10897000636624016374A400330424013304A44017
:1089800033554401930500008320C104032481046E
:1089900083244104032901048329C103032A810399
:1089A000832A4103032B0103832BC102032C810281
:1089B000832C4102032D0102832DC1011301010506
:1089C00067800000B7070001130A0001E36EF6ECB0
:1089D000130A80016FF05FED631A06009305000033
:1089E00013051000EF00C03713090500B707010099
:1089F000637AF90E9307F00F63F42701130A8000DE
:108A0000B3574901B38AFA0003C70A0013050002ED
:108A1000B384294133074701330AE540E30E0AEAEC
:108A200033194901B3DAE900B395490133D7EC00B2
:108A300093540901336BB70013850A009385040032
:108A4000EF0080369309050093850400931B09010C
:108A500013850A00EF00C03093DB0B01930505007E
:108A600013850B00EF00002D9399090193570B011B
:108A7000B3E7F90033944C0163FAA700B3872701E9
:108A800063E6270163F4A700B3872701B38AA740F1
:108A90009385040013850A00EF0000319309050057
:108AA0009385040013850A00EF00802B93050500D1
:108AB00013850B00EF00002893150B019399090112
:108AC00093D50501B3E5B90063FAA500B385250187
:108AD00063E6250163F4A500B3852501B384A540B1
:108AE0006FF09FDFB7070001130A0001E36AF9F096
:108AF000130A80016FF0DFF0E3E8D5E8B707010063
:108B000063FCF604930BF00F33B5DB00131535004F
:108B100033D7A6009777010093874771B387E700A3
:108B200083CB070093050002B38BAB00338B7541F9
:108B3000631E0B0263E4360163EACC003384CC404D
:108B4000B386D94033B58C00B384A6401305040026
:108B5000938504006FF05FE3B70700011305000180
:108B6000E3E8F6FA130580016FF09FFAB396660109
:108B7000335D7601336DDD0033D47901B39569013E
:108B800033DC7C0193540D01336CBC0013050400ED
:108B900093850400B31A6601EF000021130A050053
:108BA000938504001305040033996C01931C0D0197
:108BB000EF00001B93DC0C01130405009305050076
:108BC00013850C00EF000017131A0A0113570C014C
:108BD0003367EA00130A0400637EA7003307A70186
:108BE000130AF4FF6368A7016376A700130AE4FF82
:108BF0003307A701B309A740938504001385090033
:108C0000EF00801A93850400130405001385090002
:108C1000EF000015930505009304050013850C0073
:108C2000EF00401193150C011314040193D50501B5
:108C3000B365B4001387040063FEA500B385A501E6
:108C40001387F4FF63E8A50163F6A5001387E4FF2B
:108C5000B385A501131A0A01B70C0100336AEA00B3
:108C60001384FCFFB3778A0033F48A00B384A540F1
:108C700013850700930504002326F100135A0A0107
:108C8000EF00400B930905009305040013050A004B
:108C9000EF00400A13DC0A01930D050093050C0058
:108CA00013050A00EF0000098327C100130A05001D
:108CB00093050C0013850700EF00C0073305B501CD
:108CC00013D709013307A7006374B701330A9A0168
:108CD000B70701009387F7FF935507013377F70034
:108CE00013170701B3F7F900B3854501B307F70080
:108CF00063E6B400639EB400637CF9003386574199
:108D0000B3B7C700B385A541B385F5409307060007
:108D1000B307F9403339F900B385B440B385254131
:108D200033947501B3D767013365F400B3D565019A
:108D30006FF09FC5130605001305000093F615009C
:108D4000638406003305C50093D51500131616007D
:108D5000E39605FE678000006340050663C60506CE
:108D600013860500930505001305F0FF630C06024A
:108D700093061000637AB6006358C00013161600FD
:108D800093961600E36AB6FE1305000063E6C5007D
:108D9000B385C5403365D50093D61600135616002B
:108DA000E39606FE6780000093820000EFF05FFB11
:108DB00013850500678002003305A04063D80500D5
:108DC000B305B0406FF0DFF9B305B0409382000007
:108DD000EFF01FF93305A040678002009382000086
:108DE00063CA0500634C0500EFF09FF7138505008B
:108DF00067800200B305B040E35805FE3305A0408C
:0C8E0000EFF01FF63305B0406780020061
:02000004800278
:1000000049444C4500000000884EFEFF204EFEFF94
:100010003C4EFEFF544EFEFF644EFEFF5850FEFF66
:10002000F04FFEFF0C50FEFF2450FEFF3450FEFF49
:10003000546D7220537663008059FEFF8059FEFF95
:100040008059FEFF685AFEFF105AFEFF585AFEFF05
:100050008059FEFF8059FEFF685AFEFF105AFEFFCE
:10006000546D725100000000286E756C6C29000000
:10007000A470FEFFE073FEFFCC73FEFFE073FEFF93
:10008000E073FEFFE073FEFFE073FEFF5071FEFFC2
:10009000E073FEFFE073FEFFE870FEFF6871FEFF95
:1000A000E073FEFFF470FEFF0071FEFF0071FEFFC3
:1000B0000071FEFF0071FEFF0071FEFF0071FEFF88
:1000C0000071FEFF0071FEFF0071FEFFE073FEFF96
:1000D000E073FEFFE073FEFFE073FEFFE073FEFFE0
:1000E000E073FEFFE073FEFFE073FEFFE073FEFFD0
:1000F000E073FEFFE073FEFFE073FEFFE073FEFFC0
:10010000E073FEFFE073FEFFE073FEFFE073FEFFAF
:10011000E073FEFFE073FEFFE073FEFFE073FEFF9F
:10012000E073FEFFE073FEFFE073FEFFE073FEFF8F
:10013000E073FEFFE073FEFFE073FEFFE073FEFF7F
:10014000E073FEFFE073FEFFE073FEFFE073FEFF6F
:10015000E073FEFFE073FEFFE073FEFFE073FEFF5F
:10016000E073FEFFE073FEFFE073FEFFE073FEFF4F
:10017000A871FEFFC072FEFFE073FEFFE073FEFF9A
:10018000E073FEFFE073FEFFE073FEFFE073FEFF2F
:10019000E073FEFF9871FEFFE073FEFFE073FEFF69
:1001A0005073FEFF5C73FEFFE073FEFFE073FEFF23
:1001B000CC71FEFFE073FEFF4473FEFFE073FEFFB1
:1001C000E073FEFF8473FEFF6D69616F750A0000C6
:1001D0006D69616F75320A0068756E6772790A0021
:1001E0004572726F7220696E20416C74426C6F634D
:1001F0006B207461736B73200D0A000043686563A4
:100200006B54696D65720000416C74426C6F636B76
:100210005175657565000000464254657374310080
:100220004642546573743200000102020303030363
:100230000404040404040404050505050505050576
:100240000505050505050505060606060606060656
:10025000060606060606060606060606060606063E
:100260000606060606060606070707070707070726
:10027000070707070707070707070707070707070E
:1002800007070707070707070707070707070707FE
:1002900007070707070707070707070707070707EE
:1002A00007070707070707070808080808080808D6
:1002B00008080808080808080808080808080808BE
:1002C00008080808080808080808080808080808AE
:1002D000080808080808080808080808080808089E
:1002E000080808080808080808080808080808088E
:1002F000080808080808080808080808080808087E
:10030000080808080808080808080808080808086D
:10031000080808080808080808080808080808085D
:08032000080808080808080895
:100328001000000000000000017A5200017C010169
:100338001B0D02004C00000018000000147FFEFF97
:10034800DC05000000440E307089039507810188A0
:100358000292049305940696089709980A990B9AAD
:100368000C0370020AC144C844C944D244D344D4DB
:1003780044D544D644D744D844D944DA440E00443A
:100388000B0000005000000068000000A084FEFF81
:100398000005000000440E507488028903930599F3
:1003A8000B810192049406950796089709980A9A72
:1003B8000C9B0D0320010AC144C844C944D244D34C
:1003C80044D444D544D644D744D844D944DA44DB49
:0803D800440E00440B0000007C
:1003EC00AAAAAAAA08000000FC8F010009000000BC
:040000058000004037
:00000001FF
